 unpack

 Timestamp is 1e002ac4 (reproducible build file hash)

 Preferred load address is 0000000180000000

 Start         Length     Name                   Class
 0001:00000000 0000cb80H .text$mn                CODE
 0001:0000cb80 00000036H .text$mn$00             CODE
 0001:0000cbb6 00000092H .text$x                 CODE
 0002:00000000 000001f0H .idata$5                DATA
 0002:000001f0 00000038H .00cfg                  DATA
 0002:00000228 00000008H .CRT$XCA                DATA
 0002:00000230 00000008H .CRT$XCZ                DATA
 0002:00000238 00000008H .CRT$XIA                DATA
 0002:00000240 00000008H .CRT$XIZ                DATA
 0002:00000248 00000008H .CRT$XPA                DATA
 0002:00000250 00000008H .CRT$XPZ                DATA
 0002:00000258 00000008H .CRT$XTA                DATA
 0002:00000260 00000010H .CRT$XTZ                DATA
 0002:00000268 00000000H .gehcont$y              DATA
 0002:00000268 00000000H .gfids$y                DATA
 0002:00000270 00002e10H .rdata                  DATA
 0002:00003080 00000000H .rdata$CastGuardVftablesA DATA
 0002:00003080 00000000H .rdata$CastGuardVftablesC DATA
 0002:00003080 000001f4H .rdata$r                DATA
 0002:00003274 00000074H .rdata$voltmd           DATA
 0002:000032e8 00000300H .rdata$zzzdbg           DATA
 0002:000035e8 00000008H .rtc$IAA                DATA
 0002:000035f0 00000008H .rtc$IZZ                DATA
 0002:000035f8 00000008H .rtc$TAA                DATA
 0002:00003600 00000008H .rtc$TZZ                DATA
 0002:00003608 00000620H .xdata                  DATA
 0002:00003c28 000000f8H .xdata$x                DATA
 0002:00003d20 000001f8H .edata                  DATA
 0002:00003f18 000000dcH .idata$2                DATA
 0002:00003ff4 00000014H .idata$3                DATA
 0002:00004008 000001f0H .idata$4                DATA
 0002:000041f8 000004c8H .idata$6                DATA
 0003:00000000 00000b38H .data                   DATA
 0003:00000b38 00000080H .data$r                 DATA
 0003:00000bb8 00000028H .data$rs                DATA
 0003:00000be0 00000a30H .bss                    DATA
 0004:00000000 000007a4H .pdata                  DATA
 0005:00000000 00000060H .rsrc$01                DATA
 0005:00000060 00000310H .rsrc$02                DATA

  Address         Publics by Value              Rva+Base               Lib:Object

 0000:00000000       __AbsoluteZero             0000000000000000     <absolute>
 0000:00000000       ___safe_se_handler_count   0000000000000000     <absolute>
 0000:00000000       ___safe_se_handler_table   0000000000000000     <absolute>
 0000:00000000       __arm64x_extra_rfe_table   0000000000000000     <absolute>
 0000:00000000       __arm64x_extra_rfe_table_size 0000000000000000     <absolute>
 0000:00000000       __arm64x_native_entrypoint 0000000000000000     <absolute>
 0000:00000000       __arm64x_redirection_metadata 0000000000000000     <absolute>
 0000:00000000       __arm64x_redirection_metadata_count 0000000000000000     <absolute>
 0000:00000000       __dynamic_value_reloc_table 0000000000000000     <absolute>
 0000:00000000       __enclave_config           0000000000000000     <absolute>
 0000:00000000       __guard_check_icall_a64n_fptr 0000000000000000     <absolute>
 0000:00000000       __guard_eh_cont_count      0000000000000000     <absolute>
 0000:00000000       __guard_eh_cont_table      0000000000000000     <absolute>
 0000:00000000       __guard_fids_count         0000000000000000     <absolute>
 0000:00000000       __guard_fids_table         0000000000000000     <absolute>
 0000:00000000       __guard_iat_count          0000000000000000     <absolute>
 0000:00000000       __guard_iat_table          0000000000000000     <absolute>
 0000:00000000       __guard_longjmp_count      0000000000000000     <absolute>
 0000:00000000       __guard_longjmp_table      0000000000000000     <absolute>
 0000:00000000       __hybrid_auxiliary_delayload_iat 0000000000000000     <absolute>
 0000:00000000       __hybrid_auxiliary_delayload_iat_copy 0000000000000000     <absolute>
 0000:00000000       __hybrid_auxiliary_iat     0000000000000000     <absolute>
 0000:00000000       __hybrid_auxiliary_iat_copy 0000000000000000     <absolute>
 0000:00000000       __hybrid_code_map          0000000000000000     <absolute>
 0000:00000000       __hybrid_code_map_count    0000000000000000     <absolute>
 0000:00000000       __hybrid_image_info_bitfield 0000000000000000     <absolute>
 0000:00000000       __x64_code_ranges_to_entry_points 0000000000000000     <absolute>
 0000:00000000       __x64_code_ranges_to_entry_points_count 0000000000000000     <absolute>
 0000:00000100       __guard_flags              0000000000000100     <absolute>
 0000:00000000       __ImageBase                0000000180000000     <linker-defined>
 0001:00000000       ?getIntCount@band@@QEAAHH@Z 0000000180001000 f   bands.obj
 0001:00000104       ?getIntTotal@band@@QEAAHXZ 0000000180001104 f   bands.obj
 0001:000001b8       ?getLong@band@@QEAA_JAEAU1@_N@Z 00000001800011b8 f   bands.obj
 0001:00000204       ?getRefCommon@band@@QEAAPEAUentry@@PEAUcpindex@@_N@Z 0000000180001204 f   bands.obj
 0001:000002a8       ?initIndexes@band@@SAXPEAUunpacker@@@Z 00000001800012a8 f   bands.obj
 0001:000002fc       ?makeBands@band@@SAPEAU1@PEAUunpacker@@@Z 00000001800012fc f   bands.obj
 0001:000003b0       ?readData@band@@QEAAXH@Z   00000001800013b0 f   bands.obj
 0001:000005b8       ?setIndex@band@@QEAAXPEAUcpindex@@@Z 00000001800015b8 f   bands.obj
 0001:000005c0       ?setIndexByTag@band@@QEAAXC@Z 00000001800015c0 f   bands.obj
 0001:000005f4       ?compareTo@bytes@@QEAAHAEAU1@@Z 00000001800015f4 f   bytes.obj
 0001:00000644       ?copyFrom@bytes@@QEAAXPEBX_K1@Z 0000000180001644 f   bytes.obj
 0001:00000650       ?ensureSize@fillbytes@@QEAAX_K@Z 0000000180001650 f   bytes.obj
 0001:00000680       ?free@bytes@@QEAAXXZ       0000000180001680 f   bytes.obj
 0001:000006b4       ?freeAll@ptrlist@@QEAAXXZ  00000001800016b4 f   bytes.obj
 0001:00000718       ?grow@fillbytes@@QEAAPEAC_K@Z 0000000180001718 f   bytes.obj
 0001:000007e8       ?indexOf@ptrlist@@QEAAHPEBX@Z 00000001800017e8 f   bytes.obj
 0001:00000818       ?malloc@bytes@@QEAAX_K@Z   0000000180001818 f   bytes.obj
 0001:0000087c       ?realloc@bytes@@QEAAX_K@Z  000000018000187c f   bytes.obj
 0001:00000934       ?saveFrom@bytes@@QEAAXPEBX_K@Z 0000000180001934 f   bytes.obj
 0001:0000097c       ?writeTo@bytes@@QEAAPEACPEAC@Z 000000018000197c f   bytes.obj
 0001:000009b0       ?findByIndex@coding@@SAPEAU1@H@Z 00000001800019b0 f   coding.obj
 0001:000009d4       ?findBySpec@coding@@SAPEAU1@H@Z 00000001800019d4 f   coding.obj
 0001:00000a4c       ?findBySpec@coding@@SAPEAU1@HHHH@Z 0000000180001a4c f   coding.obj
 0001:00000a84       ?getInt@value_stream@@QEAAHXZ 0000000180001a84 f   coding.obj
 0001:00000de8       ?init@coding@@QEAAPEAU1@XZ 0000000180001de8 f   coding.obj
 0001:00000fa8       ?init@coding_method@@QEAAXAEAPEACPEAC0HPEAUcoding@@HPEAUintlist@@@Z 0000000180001fa8 f   coding.obj
 0001:00001704       ?init@value_stream@@QEAAXPEAC0PEAUcoding@@@Z 0000000180002704 f   coding.obj
 0001:00001720       ?parse@coding@@SAIAEAPEACHH@Z 0000000180002720 f   coding.obj
 0001:000017a0       ?parseMultiple@coding@@SAXAEAPEACHPEACHH@Z 00000001800027a0 f   coding.obj
 0001:00001830       ?parse_lgH@coding@@SAIAEAPEACHHH@Z 0000000180002830 f   coding.obj
 0001:000018b0       ?reset@coding_method@@QEAAXPEAUvalue_stream@@@Z 00000001800028b0 f   coding.obj
 0001:00001900       ?setCoding@value_stream@@QEAAXPEAUcoding@@@Z 0000000180002900 f   coding.obj
 0001:00001a10       ?sumInUnsignedRange@coding@@QEAAHHH@Z 0000000180002a10 f   coding.obj
 0001:00001a44       ?CallLongMethod@JNIEnv_@@QEAA_JPEAV_jobject@@PEAU_jmethodID@@ZZ 0000000180002a44 f i jni.obj
 0001:00001a68       ?CallStaticObjectMethod@JNIEnv_@@QEAAPEAV_jobject@@PEAV_jclass@@PEAU_jmethodID@@ZZ 0000000180002a68 f i jni.obj
 0001:00001a8c       ?current@unpacker@@SAPEAU1@XZ 0000000180002a8c f   jni.obj
 0001:00001c60       Java_com_sun_java_util_jar_pack_NativeUnpack_finish 0000000180002c60 f   jni.obj
 0001:00001d14       Java_com_sun_java_util_jar_pack_NativeUnpack_getNextFile 0000000180002d14 f   jni.obj
 0001:00001f24       Java_com_sun_java_util_jar_pack_NativeUnpack_getOption 0000000180002f24 f   jni.obj
 0001:00001fe4       Java_com_sun_java_util_jar_pack_NativeUnpack_getUnusedInput 0000000180002fe4 f   jni.obj
 0001:00002088       Java_com_sun_java_util_jar_pack_NativeUnpack_initIDs 0000000180003088 f   jni.obj
 0001:000021b8       Java_com_sun_java_util_jar_pack_NativeUnpack_setOption 00000001800031b8 f   jni.obj
 0001:000022a8       Java_com_sun_java_util_jar_pack_NativeUnpack_start 00000001800032a8 f   jni.obj
 0001:000023b0       ?abort@unpacker@@QEAAXPEBD@Z 00000001800033b0 f   unpack.obj
 0001:00002410       ?buildBands@attr_definitions@unpacker@@QEAAPEAPEAUband@@PEAUlayout_definition@2@@Z 0000000180003410 f   unpack.obj
 0001:00002590       ?calloc_heap@unpacker@@QEAAPEAX_K0_N1@Z 0000000180003590 f   unpack.obj
 0001:000026a0       ?checkLegacy@unpacker@@QEAAXPEBD@Z 00000001800036a0 f   unpack.obj
 0001:00002710       ?check_options@unpacker@@QEAAXXZ 0000000180003710 f   unpack.obj
 0001:00002758       ?close_output@unpacker@@QEAAPEAUfillbytes@@PEAU2@@Z 0000000180003758 f   unpack.obj
 0001:00002870       ?computeOutputIndexes@cpool@@QEAAXXZ 0000000180003870 f   unpack.obj
 0001:000028f4       ?defineLayout@attr_definitions@unpacker@@QEAAPEAUlayout_definition@2@HPEBD0@Z 00000001800038f4 f   unpack.obj
 0001:00002a14       ?ensureClass@cpool@@QEAAPEAUentry@@AEAUbytes@@@Z 0000000180003a14 f   unpack.obj
 0001:00002b00       ?ensureUtf8@cpool@@QEAAPEAUentry@@AEAUbytes@@@Z 0000000180003b00 f   unpack.obj
 0001:00002bbc       ?ensure_input@unpacker@@QEAA_N_J@Z 0000000180003bbc f   unpack.obj
 0001:00002cc8       ?ensure_put_space@unpacker@@QEAAX_K@Z 0000000180003cc8 f   unpack.obj
 0001:00002d34       ?expandSignatures@cpool@@QEAAXXZ 0000000180003d34 f   unpack.obj
 0001:00002f58       ?free@attr_definitions@unpacker@@QEAAXXZ 0000000180003f58 f i unpack.obj
 0001:00002ff4       ?free@unpacker@@QEAAXXZ    0000000180003ff4 f   unpack.obj
 0001:00003244       ?get@cpindex@@QEAAPEAUentry@@I@Z 0000000180004244 f   unpack.obj
 0001:00003268       ?getKQIndex@cpool@@QEAAPEAUcpindex@@XZ 0000000180004268 f   unpack.obj
 0001:000032fc       ?get_abort_message@unpacker@@QEAAPEBDXZ 00000001800042fc f   unpack.obj
 0001:00003304       ?get_code_header@unpacker@@QEAAXAEAH000@Z 0000000180004304 f   unpack.obj
 0001:000033d4       ?get_next_file@unpacker@@QEAAPEAUfile@1@XZ 00000001800043d4 f   unpack.obj
 0001:00003754       ?get_option@unpacker@@QEAAPEBDPEBD@Z 0000000180004754 f   unpack.obj
 0001:000038d8       ?hashTabRef@cpool@@QEAAAEAPEAUentry@@CAEAUbytes@@@Z 00000001800048d8 f   unpack.obj
 0001:000039b8       ?init@cpool@@QEAAXPEAUunpacker@@QEAH@Z 00000001800049b8 f   unpack.obj
 0001:00003b98       ?init@unpacker@@QEAAXP6A_JPEAU1@PEAX_J2@Z@Z 0000000180004b98 f   unpack.obj
 0001:00003c44       ?initGroupIndexes@cpool@@QEAAXXZ 0000000180004c44 f   unpack.obj
 0001:00003d70       ?initMemberIndexes@cpool@@QEAAXXZ 0000000180004d70 f   unpack.obj
 0001:0000406c       ?parseIntLayout@attr_definitions@unpacker@@QEAAPEBDPEBDAEAPEAUband@@C_N@Z 000000018000506c f   unpack.obj
 0001:0000419c       ?parseLayout@attr_definitions@unpacker@@QEAAPEBDPEBDAEAPEAPEAUband@@H@Z 000000018000519c f   unpack.obj
 0001:00004900       ?parseNumeral@attr_definitions@unpacker@@QEAAPEBDPEBDAEAH@Z 0000000180005900 f   unpack.obj
 0001:000049bc       ?popBody@attr_definitions@unpacker@@QEAAPEAPEAUband@@H@Z 00000001800059bc f   unpack.obj
 0001:00004a7c       ?put_label@unpacker@@QEAAXHH@Z 0000000180005a7c f   unpack.obj
 0001:00004af0       ?put_space@unpacker@@QEAAPEAC_K@Z 0000000180005af0 f   unpack.obj
 0001:00004b3c       ?put_stackmap_type@unpacker@@QEAAXXZ 0000000180005b3c f   unpack.obj
 0001:00004bd8       ?putlayout@unpacker@@QEAAXPEAPEAUband@@@Z 0000000180005bd8 f   unpack.obj
 0001:00004e14       ?putref@unpacker@@QEAAXPEAUentry@@@Z 0000000180005e14 f   unpack.obj
 0001:00004e6c       ?putref_index@unpacker@@QEAAHPEAUentry@@H@Z 0000000180005e6c f   unpack.obj
 0001:00004f1c       ?putu1ref@unpacker@@QEAAXPEAUentry@@@Z 0000000180005f1c f   unpack.obj
 0001:00004f50       ?putu2@unpacker@@QEAAXH@Z  0000000180005f50 f   unpack.obj
 0001:00004f90       ?putu4@unpacker@@QEAAXH@Z  0000000180005f90 f   unpack.obj
 0001:00004fc4       ?putu8@unpacker@@QEAAX_J@Z 0000000180005fc4 f   unpack.obj
 0001:00005024       ?readBandData@attr_definitions@unpacker@@QEAAXH@Z 0000000180006024 f   unpack.obj
 0001:00005118       ?readBandData@attr_definitions@unpacker@@QEAAXPEAPEAUband@@I@Z 0000000180006118 f   unpack.obj
 0001:0000528c       ?read_Utf8_values@unpacker@@QEAAXPEAUentry@@HC@Z 000000018000628c f i unpack.obj
 0001:000059dc       ?read_attr_defs@unpacker@@QEAAXXZ 00000001800069dc f   unpack.obj
 0001:00005d28       ?read_attrs@unpacker@@QEAAXHH@Z 0000000180006d28 f   unpack.obj
 0001:00006a08       ?read_bands@unpacker@@QEAAXXZ 0000000180007a08 f   unpack.obj
 0001:00006a90       ?read_bcs@unpacker@@QEAAXXZ 0000000180007a90 f i unpack.obj
 0001:00006e64       ?read_bootstrap_methods@unpacker@@QEAAXPEAUentry@@HC@Z 0000000180007e64 f   unpack.obj
 0001:00006ff4       ?read_classes@unpacker@@QEAAXXZ 0000000180007ff4 f   unpack.obj
 0001:0000716c       ?read_code_headers@unpacker@@QEAAXXZ 000000018000816c f   unpack.obj
 0001:00007308       ?read_cp@unpacker@@QEAAXXZ 0000000180008308 f   unpack.obj
 0001:0000767c       ?read_double_refs@unpacker@@QEAAXAEAUband@@CCPEAUentry@@HC@Z 000000018000867c f   unpack.obj
 0001:00007790       ?read_double_words@unpacker@@QEAAXAEAUband@@PEAUentry@@HCH@Z 0000000180008790 f   unpack.obj
 0001:00007848       ?read_file_header@unpacker@@QEAAXXZ 0000000180008848 f   unpack.obj
 0001:00008128       ?read_files@unpacker@@QEAAXXZ 0000000180009128 f   unpack.obj
 0001:00008248       ?read_ics@unpacker@@QEAAXXZ 0000000180009248 f   unpack.obj
 0001:000086a8       ?read_method_handle@unpacker@@QEAAXPEAUentry@@HCH@Z 00000001800096a8 f   unpack.obj
 0001:000087e4       ?read_method_type@unpacker@@QEAAXPEAUentry@@HCH@Z 00000001800097e4 f   unpack.obj
 0001:000088fc       ?read_signature_values@unpacker@@QEAAXPEAUentry@@HC@Z 00000001800098fc f   unpack.obj
 0001:00008ac8       ?read_single_refs@unpacker@@QEAAXAEAUband@@CPEAUentry@@HCH@Z 0000000180009ac8 f   unpack.obj
 0001:00008bfc       ?read_single_words@unpacker@@QEAAXAEAUband@@PEAUentry@@HCH@Z 0000000180009bfc f i unpack.obj
 0001:00008ca8       ?redirect_stdio@unpacker@@QEAAXXZ 0000000180009ca8 f   unpack.obj
 0001:00008d98       ?ref_band_for_op@unpacker@@QEAAPEAUband@@H@Z 0000000180009d98 f   unpack.obj
 0001:00008ef8       ?ref_band_for_self_op@unpacker@@QEAAPEAUband@@HAEA_NAEAH@Z 0000000180009ef8 f   unpack.obj
 0001:00008f58       ?requestOutputIndex@entry@@QEAAXAEAUcpool@@H@Z 0000000180009f58 f   unpack.obj
 0001:00008ffc       ?resetOutputIndexes@cpool@@QEAAXXZ 0000000180009ffc f   unpack.obj
 0001:00009068       ?reset_cur_classfile@unpacker@@QEAAXXZ 000000018000a068 f   unpack.obj
 0001:000090c0       ?saveTo@unpacker@@QEAAXAEAUbytes@@PEAC_K@Z 000000018000a0c0 f   unpack.obj
 0001:00009150       ?set_option@unpacker@@QEAA_NPEBD0@Z 000000018000a150 f   unpack.obj
 0001:00009300       ?start@unpacker@@QEAAXPEAX_K@Z 000000018000a300 f   unpack.obj
 0001:00009394       ?to_bci@unpacker@@QEAAII@Z 000000018000a394 f   unpack.obj
 0001:00009408       ?typeSize@entry@@QEAAHXZ   000000018000a408 f   unpack.obj
 0001:000094ac       ?write_attrs@unpacker@@QEAAHH_K@Z 000000018000a4ac f   unpack.obj
 0001:0000a0fc       ?write_bc_ops@unpacker@@QEAAXXZ 000000018000b0fc f i unpack.obj
 0001:0000aa74       ?write_bsms@unpacker@@QEAAHHH@Z 000000018000ba74 f   unpack.obj
 0001:0000ac08       ?write_classfile_head@unpacker@@QEAAXXZ 000000018000bc08 f   unpack.obj
 0001:0000adf0       ?write_classfile_tail@unpacker@@QEAAXXZ 000000018000bdf0 f   unpack.obj
 0001:0000b0d8       ?write_code@unpacker@@QEAAXXZ 000000018000c0d8 f i unpack.obj
 0001:0000b2f4       ?write_ics@unpacker@@QEAAHHH@Z 000000018000c2f4 f   unpack.obj
 0001:0000b6d4       ?write_members@unpacker@@QEAAXHH@Z 000000018000c6d4 f   unpack.obj
 0001:0000b84c       __local_stdio_printf_options 000000018000c84c f i unpack.obj
 0001:0000b854       _snprintf                  000000018000c854 f i unpack.obj
 0001:0000b8ac       fprintf                    000000018000c8ac f i unpack.obj
 0001:0000b8f0       outputEntry_cmp            000000018000c8f0 f   unpack.obj
 0001:0000b95c       raw_address_cmp            000000018000c95c f   unpack.obj
 0001:0000b970       sprintf                    000000018000c970 f i unpack.obj
 0001:0000b9c8       ?must_calloc@@YAPEAX_K0@Z  000000018000c9c8 f   utils.obj
 0001:0000ba28       ?unpack_abort@@YAXPEBDPEAUunpacker@@@Z 000000018000ca28 f   utils.obj
 0001:0000ba80       ?unpack_aborting@@YA_NPEAUunpacker@@@Z 000000018000ca80 f   utils.obj
 0001:0000bac4       ?free@gunzip@@QEAAXXZ      000000018000cac4 f   zip.obj
 0001:0000bac4       _guard_check_icall_nop     000000018000cac4 f   MSVCRT:guard_support.obj
 0001:0000bac8       ?init@jar@@QEAAXPEAUunpacker@@@Z 000000018000cac8 f   zip.obj
 0001:0000baf6       JNU_ThrowIOException       000000018000caf6 f   java:java.dll
 0001:0000bafc       __GSHandlerCheck           000000018000cafc f   MSVCRT:gshandler.obj
 0001:0000bb1c       __GSHandlerCheckCommon     000000018000cb1c f   MSVCRT:gshandler.obj
 0001:0000bb90       __security_check_cookie    000000018000cb90 f   MSVCRT:amdsecgs.obj
 0001:0000bbb0       ??2@YAPEAX_K@Z             000000018000cbb0 f   MSVCRT:new_scalar.obj
 0001:0000bbec       ??3@YAXPEAX_K@Z            000000018000cbec f   MSVCRT:delete_scalar_size.obj
 0001:0000bc10       __chkstk                   000000018000cc10 f   MSVCRT:chkstk.obj
 0001:0000bc10       _alloca_probe              000000018000cc10 f   MSVCRT:chkstk.obj
 0001:0000bf80       _DllMainCRTStartup         000000018000cf80 f   MSVCRT:dll_dllmain.obj
 0001:0000bfc0       __raise_securityfailure    000000018000cfc0 f   MSVCRT:gs_report.obj
 0001:0000bff4       __report_gsfailure         000000018000cff4 f   MSVCRT:gs_report.obj
 0001:0000c13c       ??0bad_alloc@std@@QEAA@AEBV01@@Z 000000018000d13c f i MSVCRT:throw_bad_alloc.obj
 0001:0000c178       ??0bad_alloc@std@@QEAA@XZ  000000018000d178 f i MSVCRT:throw_bad_alloc.obj
 0001:0000c198       ??0bad_array_new_length@std@@QEAA@AEBV01@@Z 000000018000d198 f i MSVCRT:throw_bad_alloc.obj
 0001:0000c1d4       ??0bad_array_new_length@std@@QEAA@XZ 000000018000d1d4 f i MSVCRT:throw_bad_alloc.obj
 0001:0000c1f4       ??0exception@std@@QEAA@AEBV01@@Z 000000018000d1f4 f i MSVCRT:throw_bad_alloc.obj
 0001:0000c228       ??1bad_alloc@std@@UEAA@XZ  000000018000d228 f i MSVCRT:throw_bad_alloc.obj
 0001:0000c228       ??1bad_array_new_length@std@@UEAA@XZ 000000018000d228 f i MSVCRT:throw_bad_alloc.obj
 0001:0000c23c       ??_Ebad_alloc@std@@UEAAPEAXI@Z 000000018000d23c f i MSVCRT:throw_bad_alloc.obj
 0001:0000c23c       ??_Ebad_array_new_length@std@@UEAAPEAXI@Z 000000018000d23c f i MSVCRT:throw_bad_alloc.obj
 0001:0000c23c       ??_Eexception@std@@UEAAPEAXI@Z 000000018000d23c f i MSVCRT:throw_bad_alloc.obj
 0001:0000c23c       ??_Gbad_alloc@std@@UEAAPEAXI@Z 000000018000d23c f i MSVCRT:throw_bad_alloc.obj
 0001:0000c23c       ??_Gbad_array_new_length@std@@UEAAPEAXI@Z 000000018000d23c f i MSVCRT:throw_bad_alloc.obj
 0001:0000c23c       ??_Gexception@std@@UEAAPEAXI@Z 000000018000d23c f i MSVCRT:throw_bad_alloc.obj
 0001:0000c280       ?__scrt_throw_std_bad_alloc@@YAXXZ 000000018000d280 f   MSVCRT:throw_bad_alloc.obj
 0001:0000c2a0       ?__scrt_throw_std_bad_array_new_length@@YAXXZ 000000018000d2a0 f   MSVCRT:throw_bad_alloc.obj
 0001:0000c2c0       ?what@exception@std@@UEBAPEBDXZ 000000018000d2c0 f i MSVCRT:throw_bad_alloc.obj
 0001:0000c2d4       ??3@YAXPEAX@Z              000000018000d2d4 f   MSVCRT:delete_scalar.obj
 0001:0000c2dc       __security_init_cookie     000000018000d2dc f   MSVCRT:gs_support.obj
 0001:0000c388       DllMain                    000000018000d388 f   MSVCRT:dll_dllmain_stub.obj
 0001:0000c3ac       ?__scrt_initialize_type_info@@YAXXZ 000000018000d3ac f   MSVCRT:tncleanup.obj
 0001:0000c3bc       ?__scrt_uninitialize_type_info@@YAXXZ 000000018000d3bc f   MSVCRT:tncleanup.obj
 0001:0000c3c8       __local_stdio_scanf_options 000000018000d3c8 f i MSVCRT:default_local_stdio_options.obj
 0001:0000c3d0       __scrt_initialize_default_local_stdio_options 000000018000d3d0 f   MSVCRT:default_local_stdio_options.obj
 0001:0000c3ec       __scrt_acquire_startup_lock 000000018000d3ec f   MSVCRT:utility.obj
 0001:0000c428       __scrt_dllmain_after_initialize_c 000000018000d428 f   MSVCRT:utility.obj
 0001:0000c45c       __scrt_dllmain_before_initialize_c 000000018000d45c f   MSVCRT:utility.obj
 0001:0000c474       __scrt_dllmain_crt_thread_attach 000000018000d474 f   MSVCRT:utility.obj
 0001:0000c49c       __scrt_dllmain_crt_thread_detach 000000018000d49c f   MSVCRT:utility.obj
 0001:0000c4b4       __scrt_dllmain_exception_filter 000000018000d4b4 f   MSVCRT:utility.obj
 0001:0000c514       __scrt_dllmain_uninitialize_c 000000018000d514 f   MSVCRT:utility.obj
 0001:0000c544       __scrt_dllmain_uninitialize_critical 000000018000d544 f   MSVCRT:utility.obj
 0001:0000c558       __scrt_initialize_crt      000000018000d558 f   MSVCRT:utility.obj
 0001:0000c5a4       __scrt_initialize_onexit_tables 000000018000d5a4 f   MSVCRT:utility.obj
 0001:0000c630       __scrt_is_nonwritable_in_current_image 000000018000d630 f   MSVCRT:utility.obj
 0001:0000c6c8       __scrt_release_startup_lock 000000018000d6c8 f   MSVCRT:utility.obj
 0001:0000c6ec       __scrt_uninitialize_crt    000000018000d6ec f   MSVCRT:utility.obj
 0001:0000c718       __scrt_get_dyn_tls_init_callback 000000018000d718 f   MSVCRT:dyn_tls_init.obj
 0001:0000c720       __crt_debugger_hook        000000018000d720 f   MSVCRT:utility_desktop.obj
 0001:0000c728       __scrt_fastfail            000000018000d728 f   MSVCRT:utility_desktop.obj
 0001:0000c874       _RTC_Initialize            000000018000d874 f   MSVCRT:initsect.obj
 0001:0000c8b0       _RTC_Terminate             000000018000d8b0 f   MSVCRT:initsect.obj
 0001:0000c8ec       ??_Etype_info@@UEAAPEAXI@Z 000000018000d8ec f i MSVCRT:std_type_info_static.obj
 0001:0000c8ec       ??_Gtype_info@@UEAAPEAXI@Z 000000018000d8ec f i MSVCRT:std_type_info_static.obj
 0001:0000c918       __isa_available_init       000000018000d918 f   MSVCRT:cpu_disp.obj
 0001:0000cac4       _get_startup_argv_mode     000000018000dac4 f   MSVCRT:argv_mode.obj
 0001:0000cacc       __scrt_is_ucrt_dll_in_use  000000018000dacc f   MSVCRT:ucrt_detection.obj
 0001:0000cae0       memcmp                     000000018000dae0 f   vcruntime:VCRUNTIME140.dll
 0001:0000cae6       memcpy                     000000018000dae6 f   vcruntime:VCRUNTIME140.dll
 0001:0000caec       memset                     000000018000daec f   vcruntime:VCRUNTIME140.dll
 0001:0000caf2       strchr                     000000018000daf2 f   vcruntime:VCRUNTIME140.dll
 0001:0000caf8       __C_specific_handler       000000018000daf8 f   vcruntime:VCRUNTIME140.dll
 0001:0000cafe       __std_exception_copy       000000018000dafe f   vcruntime:VCRUNTIME140.dll
 0001:0000cb04       __std_exception_destroy    000000018000db04 f   vcruntime:VCRUNTIME140.dll
 0001:0000cb0a       _CxxThrowException         000000018000db0a f   vcruntime:VCRUNTIME140.dll
 0001:0000cb10       __std_type_info_destroy_list 000000018000db10 f   vcruntime:VCRUNTIME140.dll
 0001:0000cb16       free                       000000018000db16 f   ucrt:api-ms-win-crt-heap-l1-1-0.dll
 0001:0000cb1c       strcat                     000000018000db1c f   ucrt:api-ms-win-crt-string-l1-1-0.dll
 0001:0000cb22       strcmp                     000000018000db22 f   ucrt:api-ms-win-crt-string-l1-1-0.dll
 0001:0000cb28       strlen                     000000018000db28 f   ucrt:api-ms-win-crt-string-l1-1-0.dll
 0001:0000cb2e       _callnewh                  000000018000db2e f   ucrt:api-ms-win-crt-heap-l1-1-0.dll
 0001:0000cb34       malloc                     000000018000db34 f   ucrt:api-ms-win-crt-heap-l1-1-0.dll
 0001:0000cb3a       _initterm                  000000018000db3a f   ucrt:api-ms-win-crt-runtime-l1-1-0.dll
 0001:0000cb40       _initterm_e                000000018000db40 f   ucrt:api-ms-win-crt-runtime-l1-1-0.dll
 0001:0000cb46       _seh_filter_dll            000000018000db46 f   ucrt:api-ms-win-crt-runtime-l1-1-0.dll
 0001:0000cb4c       _configure_narrow_argv     000000018000db4c f   ucrt:api-ms-win-crt-runtime-l1-1-0.dll
 0001:0000cb52       _initialize_narrow_environment 000000018000db52 f   ucrt:api-ms-win-crt-runtime-l1-1-0.dll
 0001:0000cb58       _initialize_onexit_table   000000018000db58 f   ucrt:api-ms-win-crt-runtime-l1-1-0.dll
 0001:0000cb5e       _execute_onexit_table      000000018000db5e f   ucrt:api-ms-win-crt-runtime-l1-1-0.dll
 0001:0000cb64       _cexit                     000000018000db64 f   ucrt:api-ms-win-crt-runtime-l1-1-0.dll
 0001:0000cb6c       __acrt_initialize          000000018000db6c f   MSVCRT:ucrt_stubs.obj
 0001:0000cb6c       __acrt_thread_attach       000000018000db6c f   MSVCRT:ucrt_stubs.obj
 0001:0000cb6c       __acrt_thread_detach       000000018000db6c f   MSVCRT:ucrt_stubs.obj
 0001:0000cb6c       __acrt_uninitialize        000000018000db6c f   MSVCRT:ucrt_stubs.obj
 0001:0000cb6c       __acrt_uninitialize_critical 000000018000db6c f   MSVCRT:ucrt_stubs.obj
 0001:0000cb6c       __scrt_stub_for_acrt_initialize 000000018000db6c f   MSVCRT:ucrt_stubs.obj
 0001:0000cb6c       __scrt_stub_for_acrt_thread_attach 000000018000db6c f   MSVCRT:ucrt_stubs.obj
 0001:0000cb6c       __scrt_stub_for_acrt_thread_detach 000000018000db6c f   MSVCRT:ucrt_stubs.obj
 0001:0000cb6c       __scrt_stub_for_acrt_uninitialize 000000018000db6c f   MSVCRT:ucrt_stubs.obj
 0001:0000cb6c       __scrt_stub_for_acrt_uninitialize_critical 000000018000db6c f   MSVCRT:ucrt_stubs.obj
 0001:0000cb6c       __vcrt_initialize          000000018000db6c f   MSVCRT:ucrt_stubs.obj
 0001:0000cb6c       __vcrt_thread_attach       000000018000db6c f   MSVCRT:ucrt_stubs.obj
 0001:0000cb6c       __vcrt_thread_detach       000000018000db6c f   MSVCRT:ucrt_stubs.obj
 0001:0000cb6c       __vcrt_uninitialize        000000018000db6c f   MSVCRT:ucrt_stubs.obj
 0001:0000cb6c       __vcrt_uninitialize_critical 000000018000db6c f   MSVCRT:ucrt_stubs.obj
 0001:0000cb70       __scrt_stub_for_is_c_termination_complete 000000018000db70 f   MSVCRT:ucrt_stubs.obj
 0001:0000cb70       _is_c_termination_complete 000000018000db70 f   MSVCRT:ucrt_stubs.obj
 0001:0000cb90       _guard_dispatch_icall_nop  000000018000db90 f   MSVCRT:guard_dispatch.obj
 0001:0000cbb0       _guard_xfg_dispatch_icall_nop 000000018000dbb0 f   MSVCRT:guard_xfg_dispatch.obj
 0002:00000000       __imp_IsDebuggerPresent    000000018000e000     kernel32:KERNEL32.dll
 0002:00000008       __imp_InitializeSListHead  000000018000e008     kernel32:KERNEL32.dll
 0002:00000010       __imp_RtlCaptureContext    000000018000e010     kernel32:KERNEL32.dll
 0002:00000018       __imp_RtlLookupFunctionEntry 000000018000e018     kernel32:KERNEL32.dll
 0002:00000020       __imp_RtlVirtualUnwind     000000018000e020     kernel32:KERNEL32.dll
 0002:00000028       __imp_UnhandledExceptionFilter 000000018000e028     kernel32:KERNEL32.dll
 0002:00000030       __imp_SetUnhandledExceptionFilter 000000018000e030     kernel32:KERNEL32.dll
 0002:00000038       __imp_GetCurrentProcess    000000018000e038     kernel32:KERNEL32.dll
 0002:00000040       __imp_TerminateProcess     000000018000e040     kernel32:KERNEL32.dll
 0002:00000048       __imp_IsProcessorFeaturePresent 000000018000e048     kernel32:KERNEL32.dll
 0002:00000050       __imp_QueryPerformanceCounter 000000018000e050     kernel32:KERNEL32.dll
 0002:00000058       __imp_GetCurrentProcessId  000000018000e058     kernel32:KERNEL32.dll
 0002:00000060       __imp_GetCurrentThreadId   000000018000e060     kernel32:KERNEL32.dll
 0002:00000068       __imp_GetSystemTimeAsFileTime 000000018000e068     kernel32:KERNEL32.dll
 0002:00000070       __imp_DisableThreadLibraryCalls 000000018000e070     kernel32:KERNEL32.dll
 0002:00000078       \177KERNEL32_NULL_THUNK_DATA 000000018000e078     kernel32:KERNEL32.dll
 0002:00000080       __imp___std_type_info_destroy_list 000000018000e080     vcruntime:VCRUNTIME140.dll
 0002:00000088       __imp__CxxThrowException   000000018000e088     vcruntime:VCRUNTIME140.dll
 0002:00000090       __imp_memcmp               000000018000e090     vcruntime:VCRUNTIME140.dll
 0002:00000098       __imp_memcpy               000000018000e098     vcruntime:VCRUNTIME140.dll
 0002:000000a0       __imp_memset               000000018000e0a0     vcruntime:VCRUNTIME140.dll
 0002:000000a8       __imp_strchr               000000018000e0a8     vcruntime:VCRUNTIME140.dll
 0002:000000b0       __imp___C_specific_handler 000000018000e0b0     vcruntime:VCRUNTIME140.dll
 0002:000000b8       __imp___std_exception_copy 000000018000e0b8     vcruntime:VCRUNTIME140.dll
 0002:000000c0       __imp___std_exception_destroy 000000018000e0c0     vcruntime:VCRUNTIME140.dll
 0002:000000c8       \177VCRUNTIME140_NULL_THUNK_DATA 000000018000e0c8     vcruntime:VCRUNTIME140.dll
 0002:000000d0       __imp_atoi                 000000018000e0d0     ucrt:api-ms-win-crt-convert-l1-1-0.dll
 0002:000000d8       \177api-ms-win-crt-convert-l1-1-0_NULL_THUNK_DATA 000000018000e0d8     ucrt:api-ms-win-crt-convert-l1-1-0.dll
 0002:000000e0       __imp_free                 000000018000e0e0     ucrt:api-ms-win-crt-heap-l1-1-0.dll
 0002:000000e8       __imp_realloc              000000018000e0e8     ucrt:api-ms-win-crt-heap-l1-1-0.dll
 0002:000000f0       __imp_calloc               000000018000e0f0     ucrt:api-ms-win-crt-heap-l1-1-0.dll
 0002:000000f8       __imp__callnewh            000000018000e0f8     ucrt:api-ms-win-crt-heap-l1-1-0.dll
 0002:00000100       __imp_malloc               000000018000e100     ucrt:api-ms-win-crt-heap-l1-1-0.dll
 0002:00000108       \177api-ms-win-crt-heap-l1-1-0_NULL_THUNK_DATA 000000018000e108     ucrt:api-ms-win-crt-heap-l1-1-0.dll
 0002:00000110       __imp__initterm_e          000000018000e110     ucrt:api-ms-win-crt-runtime-l1-1-0.dll
 0002:00000118       __imp__seh_filter_dll      000000018000e118     ucrt:api-ms-win-crt-runtime-l1-1-0.dll
 0002:00000120       __imp__configure_narrow_argv 000000018000e120     ucrt:api-ms-win-crt-runtime-l1-1-0.dll
 0002:00000128       __imp__cexit               000000018000e128     ucrt:api-ms-win-crt-runtime-l1-1-0.dll
 0002:00000130       __imp__execute_onexit_table 000000018000e130     ucrt:api-ms-win-crt-runtime-l1-1-0.dll
 0002:00000138       __imp__initterm            000000018000e138     ucrt:api-ms-win-crt-runtime-l1-1-0.dll
 0002:00000140       __imp_abort                000000018000e140     ucrt:api-ms-win-crt-runtime-l1-1-0.dll
 0002:00000148       __imp__initialize_onexit_table 000000018000e148     ucrt:api-ms-win-crt-runtime-l1-1-0.dll
 0002:00000150       __imp__initialize_narrow_environment 000000018000e150     ucrt:api-ms-win-crt-runtime-l1-1-0.dll
 0002:00000158       \177api-ms-win-crt-runtime-l1-1-0_NULL_THUNK_DATA 000000018000e158     ucrt:api-ms-win-crt-runtime-l1-1-0.dll
 0002:00000160       __imp___stdio_common_vsprintf 000000018000e160     ucrt:api-ms-win-crt-stdio-l1-1-0.dll
 0002:00000168       __imp___stdio_common_vfprintf 000000018000e168     ucrt:api-ms-win-crt-stdio-l1-1-0.dll
 0002:00000170       __imp_fopen                000000018000e170     ucrt:api-ms-win-crt-stdio-l1-1-0.dll
 0002:00000178       __imp___acrt_iob_func      000000018000e178     ucrt:api-ms-win-crt-stdio-l1-1-0.dll
 0002:00000180       \177api-ms-win-crt-stdio-l1-1-0_NULL_THUNK_DATA 000000018000e180     ucrt:api-ms-win-crt-stdio-l1-1-0.dll
 0002:00000188       __imp_strcmp               000000018000e188     ucrt:api-ms-win-crt-string-l1-1-0.dll
 0002:00000190       __imp_strlen               000000018000e190     ucrt:api-ms-win-crt-string-l1-1-0.dll
 0002:00000198       __imp_strncat              000000018000e198     ucrt:api-ms-win-crt-string-l1-1-0.dll
 0002:000001a0       __imp_strcat               000000018000e1a0     ucrt:api-ms-win-crt-string-l1-1-0.dll
 0002:000001a8       \177api-ms-win-crt-string-l1-1-0_NULL_THUNK_DATA 000000018000e1a8     ucrt:api-ms-win-crt-string-l1-1-0.dll
 0002:000001b0       __imp__time64              000000018000e1b0     ucrt:api-ms-win-crt-time-l1-1-0.dll
 0002:000001b8       \177api-ms-win-crt-time-l1-1-0_NULL_THUNK_DATA 000000018000e1b8     ucrt:api-ms-win-crt-time-l1-1-0.dll
 0002:000001c0       __imp_qsort                000000018000e1c0     ucrt:api-ms-win-crt-utility-l1-1-0.dll
 0002:000001c8       \177api-ms-win-crt-utility-l1-1-0_NULL_THUNK_DATA 000000018000e1c8     ucrt:api-ms-win-crt-utility-l1-1-0.dll
 0002:000001d0       __imp_JNU_ThrowIOException 000000018000e1d0     java:java.dll
 0002:000001d8       \177java_NULL_THUNK_DATA   000000018000e1d8     java:java.dll
 0002:000001e0       __imp_JNI_GetCreatedJavaVMs 000000018000e1e0     jvm:jvm.dll
 0002:000001e8       \177jvm_NULL_THUNK_DATA    000000018000e1e8     jvm:jvm.dll
 0002:000001f0       __guard_check_icall_fptr   000000018000e1f0     MSVCRT:guard_support.obj
 0002:000001f8       __guard_xfg_check_icall_fptr 000000018000e1f8     MSVCRT:guard_support.obj
 0002:00000200       __guard_dispatch_icall_fptr 000000018000e200     MSVCRT:guard_support.obj
 0002:00000208       __guard_xfg_dispatch_icall_fptr 000000018000e208     MSVCRT:guard_support.obj
 0002:00000210       __guard_xfg_table_dispatch_icall_fptr 000000018000e210     MSVCRT:guard_support.obj
 0002:00000218       __castguard_check_failure_os_handled_fptr 000000018000e218     MSVCRT:guard_support.obj
 0002:00000220       __guard_memcpy_fptr        000000018000e220     vcruntime:softmemtag.obj
 0002:00000228       __xc_a                     000000018000e228     MSVCRT:initializers.obj
 0002:00000230       __xc_z                     000000018000e230     MSVCRT:initializers.obj
 0002:00000238       __xi_a                     000000018000e238     MSVCRT:initializers.obj
 0002:00000240       __xi_z                     000000018000e240     MSVCRT:initializers.obj
 0002:00000248       __xp_a                     000000018000e248     MSVCRT:initializers.obj
 0002:00000250       __xp_z                     000000018000e250     MSVCRT:initializers.obj
 0002:00000258       __xt_a                     000000018000e258     MSVCRT:initializers.obj
 0002:00000260       __xt_z                     000000018000e260     MSVCRT:initializers.obj
 0002:00001110       ??_C@_0P@NFDCFGCL@cp_Utf8_prefix@ 000000018000f110     bands.obj
 0002:00001120       ??_C@_0P@LOHPAGNO@cp_Utf8_suffix@ 000000018000f120     bands.obj
 0002:00001130       ??_C@_0O@IHLLKPBK@cp_Utf8_chars@ 000000018000f130     bands.obj
 0002:00001140       ??_C@_0BD@EOIEJGOP@cp_Utf8_big_suffix@ 000000018000f140     bands.obj
 0002:00001158       ??_C@_0BC@HDLINKIK@cp_Utf8_big_chars@ 000000018000f158     bands.obj
 0002:0000116c       ??_C@_06IGKKGOEN@cp_Int@   000000018000f16c     bands.obj
 0002:00001178       ??_C@_08OBBFNHHD@cp_Float@ 000000018000f178     bands.obj
 0002:00001188       ??_C@_0L@HNFJMOEO@cp_Long_hi@ 000000018000f188     bands.obj
 0002:00001198       ??_C@_0L@CMAKMBBE@cp_Long_lo@ 000000018000f198     bands.obj
 0002:000011a8       ??_C@_0N@CPNNOOPC@cp_Double_hi@ 000000018000f1a8     bands.obj
 0002:000011b8       ??_C@_0N@HOIOOBKI@cp_Double_lo@ 000000018000f1b8     bands.obj
 0002:000011c8       ??_C@_09HFEHKGNE@cp_String@ 000000018000f1c8     bands.obj
 0002:000011d8       ??_C@_08BOENACK@cp_Class@  000000018000f1d8     bands.obj
 0002:000011e8       ??_C@_0BC@FENMLAPO@cp_Signature_form@ 000000018000f1e8     bands.obj
 0002:00001200       ??_C@_0BF@MEOEAPGK@cp_Signature_classes@ 000000018000f200     bands.obj
 0002:00001218       ??_C@_0O@JHMEINNJ@cp_Descr_name@ 000000018000f218     bands.obj
 0002:00001228       ??_C@_0O@DMMHENKJ@cp_Descr_type@ 000000018000f228     bands.obj
 0002:00001238       ??_C@_0P@EEAFDJFH@cp_Field_class@ 000000018000f238     bands.obj
 0002:00001248       ??_C@_0O@FCFAPCDP@cp_Field_desc@ 000000018000f248     bands.obj
 0002:00001258       ??_C@_0BA@LDOOFFKI@cp_Method_class@ 000000018000f258     bands.obj
 0002:00001268       ??_C@_0P@NLGLFAKL@cp_Method_desc@ 000000018000f268     bands.obj
 0002:00001278       ??_C@_0BB@IIGJKIIK@cp_Imethod_class@ 000000018000f278     bands.obj
 0002:00001290       ??_C@_0BA@DCLGLKIL@cp_Imethod_desc@ 000000018000f290     bands.obj
 0002:000012a0       ??_C@_0BI@NIJEEAN@cp_MethodHandle_refkind@ 000000018000f2a0     bands.obj
 0002:000012b8       ??_C@_0BH@NKNCKAEO@cp_MethodHandle_member@ 000000018000f2b8     bands.obj
 0002:000012d0       ??_C@_0O@NHPECHNH@cp_MethodType@ 000000018000f2d0     bands.obj
 0002:000012e0       ??_C@_0BH@NPCIPIPL@cp_BootstrapMethod_ref@ 000000018000f2e0     bands.obj
 0002:000012f8       ??_C@_0BN@DJLEBMBH@cp_BootstrapMethod_arg_count@ 000000018000f2f8     bands.obj
 0002:00001318       ??_C@_0BH@JNPGIEDO@cp_BootstrapMethod_arg@ 000000018000f318     bands.obj
 0002:00001330       ??_C@_0BG@CIPOMBAC@cp_InvokeDynamic_spec@ 000000018000f330     bands.obj
 0002:00001348       ??_C@_0BG@IFFCPCPP@cp_InvokeDynamic_desc@ 000000018000f348     bands.obj
 0002:00001360       ??_C@_0BI@KJJNKCHD@attr_definition_headers@ 000000018000f360     bands.obj
 0002:00001378       ??_C@_0BF@EEAHHHEA@attr_definition_name@ 000000018000f378     bands.obj
 0002:00001390       ??_C@_0BH@EKDDDJNL@attr_definition_layout@ 000000018000f390     bands.obj
 0002:000013a8       ??_C@_0O@HJMNFDHJ@ic_this_class@ 000000018000f3a8     bands.obj
 0002:000013b8       ??_C@_08CKLAPDFF@ic_flags@ 000000018000f3b8     bands.obj
 0002:000013c8       ??_C@_0P@MGLGIOLC@ic_outer_class@ 000000018000f3c8     bands.obj
 0002:000013d8       ??_C@_07OPOCOJIH@ic_name@  000000018000f3d8     bands.obj
 0002:000013e0       ??_C@_0L@GONOGKKN@class_this@ 000000018000f3e0     bands.obj
 0002:000013f0       ??_C@_0M@FMPLOBH@class_super@ 000000018000f3f0     bands.obj
 0002:00001400       ??_C@_0BG@ELABOHHB@class_interface_count@ 000000018000f400     bands.obj
 0002:00001418       ??_C@_0BA@GDKGLIFF@class_interface@ 000000018000f418     bands.obj
 0002:00001428       ??_C@_0BC@GLACLOBG@class_field_count@ 000000018000f428     bands.obj
 0002:00001440       ??_C@_0BD@MFLGOFPO@class_method_count@ 000000018000f440     bands.obj
 0002:00001458       ??_C@_0M@IINMAGFA@field_descr@ 000000018000f458     bands.obj
 0002:00001468       ??_C@_0P@LDBPJHCP@field_flags_hi@ 000000018000f468     bands.obj
 0002:00001478       ??_C@_0P@OCEMJIHF@field_flags_lo@ 000000018000f478     bands.obj
 0002:00001488       ??_C@_0BB@GJGJJLKK@field_attr_count@ 000000018000f488     bands.obj
 0002:000014a0       ??_C@_0BD@LLAABMND@field_attr_indexes@ 000000018000f4a0     bands.obj
 0002:000014b8       ??_C@_0BB@LHINHPHH@field_attr_calls@ 000000018000f4b8     bands.obj
 0002:000014d0       ??_C@_0BH@NKCAAIDC@field_ConstantValue_KQ@ 000000018000f4d0     bands.obj
 0002:000014e8       ??_C@_0BD@HMEKDNDB@field_Signature_RS@ 000000018000f4e8     bands.obj
 0002:00001500       ??_C@_0BF@KACJMLOM@field_metadata_bands@ 000000018000f500     bands.obj
 0002:00001518       ??_C@_0BB@NIMLDFOB@field_attr_bands@ 000000018000f518     bands.obj
 0002:00001530       ??_C@_0N@GLCNNANE@method_descr@ 000000018000f530     bands.obj
 0002:00001540       ??_C@_0BA@EIPLIEID@method_flags_hi@ 000000018000f540     bands.obj
 0002:00001550       ??_C@_0BA@BJKIILNJ@method_flags_lo@ 000000018000f550     bands.obj
 0002:00001560       ??_C@_0BC@OPGFNCHF@method_attr_count@ 000000018000f560     bands.obj
 0002:00001578       ??_C@_0BE@LCKALKDL@method_attr_indexes@ 000000018000f578     bands.obj
 0002:00001590       ??_C@_0BC@DBIBDGKI@method_attr_calls@ 000000018000f590     bands.obj
 0002:000015a8       ??_C@_0BE@HAIBKECN@method_Exceptions_N@ 000000018000f5a8     bands.obj
 0002:000015c0       ??_C@_0BF@ILMHJLAD@method_Exceptions_RC@ 000000018000f5c0     bands.obj
 0002:000015d8       ??_C@_0BE@HFOKJLNJ@method_Signature_RS@ 000000018000f5d8     bands.obj
 0002:000015f0       ??_C@_0BG@JDLLNHF@method_metadata_bands@ 000000018000f5f0     bands.obj
 0002:00001608       ??_C@_0BL@MNBFAABE@method_MethodParameters_NB@ 000000018000f608     bands.obj
 0002:00001628       ??_C@_0CB@POGNKHAK@method_MethodParameters_name_RU@ 000000018000f628     bands.obj
 0002:00001650       ??_C@_0CA@HDKLJONB@method_MethodParameters_flag_FH@ 000000018000f650     bands.obj
 0002:00001670       ??_C@_0BC@FOMHHMDO@method_attr_bands@ 000000018000f670     bands.obj
 0002:00001688       ??_C@_0P@DNMDIOJK@class_flags_hi@ 000000018000f688     bands.obj
 0002:00001698       ??_C@_0P@GMJAIBMA@class_flags_lo@ 000000018000f698     bands.obj
 0002:000016a8       ??_C@_0BB@JELAOHEL@class_attr_count@ 000000018000f6a8     bands.obj
 0002:000016c0       ??_C@_0BD@KFNGBOLA@class_attr_indexes@ 000000018000f6c0     bands.obj
 0002:000016d8       ??_C@_0BB@EKFEADJG@class_attr_calls@ 000000018000f6d8     bands.obj
 0002:000016f0       ??_C@_0BF@MJNFEGEM@class_SourceFile_RUN@ 000000018000f6f0     bands.obj
 0002:00001708       ??_C@_0BJ@CCGEELON@class_EnclosingMethod_RC@ 000000018000f708     bands.obj
 0002:00001728       ??_C@_0BK@LFCMIOIA@class_EnclosingMethod_RDN@ 000000018000f728     bands.obj
 0002:00001748       ??_C@_0BD@GCJMDPFC@class_Signature_RS@ 000000018000f748     bands.obj
 0002:00001760       ??_C@_0BF@PHIMHC@class_metadata_bands@ 000000018000f760     bands.obj
 0002:00001778       ??_C@_0BF@PGJMDHG@class_InnerClasses_N@ 000000018000f778     bands.obj
 0002:00001790       ??_C@_0BG@HHABPLBI@class_InnerClasses_RC@ 000000018000f790     bands.obj
 0002:000017a8       ??_C@_0BF@MHLAEJHO@class_InnerClasses_F@ 000000018000f7a8     bands.obj
 0002:000017c0       ??_C@_0BN@FANFKEPF@class_InnerClasses_outer_RCN@ 000000018000f7c0     bands.obj
 0002:000017e0       ??_C@_0BM@CHKHAMMI@class_InnerClasses_name_RUN@ 000000018000f7e0     bands.obj
 0002:00001800       ??_C@_0CA@LBNJCLO@class_ClassFile_version_minor_H@ 000000018000f800     bands.obj
 0002:00001820       ??_C@_0CA@KDGDJOMP@class_ClassFile_version_major_H@ 000000018000f820     bands.obj
 0002:00001840       ??_C@_0BB@CFBCEJAA@class_attr_bands@ 000000018000f840     bands.obj
 0002:00001858       ??_C@_0N@EJFJBMLJ@code_headers@ 000000018000f858     bands.obj
 0002:00001868       ??_C@_0P@DPBEANCA@code_max_stack@ 000000018000f868     bands.obj
 0002:00001878       ??_C@_0BD@OBGMDNFJ@code_max_na_locals@ 000000018000f878     bands.obj
 0002:00001890       ??_C@_0BD@OMMDBBC@code_handler_count@ 000000018000f890     bands.obj
 0002:000018a8       ??_C@_0BF@NAEEIJON@code_handler_start_P@ 000000018000f8a8     bands.obj
 0002:000018c0       ??_C@_0BE@GIJMHOG@code_handler_end_PO@ 000000018000f8c0     bands.obj
 0002:000018d8       ??_C@_0BG@GJGNOMGM@code_handler_catch_PO@ 000000018000f8d8     bands.obj
 0002:000018f0       ??_C@_0BH@ECFPKFHF@code_handler_class_RCN@ 000000018000f8f0     bands.obj
 0002:00001908       ??_C@_0O@PKFJGJJN@code_flags_hi@ 000000018000f908     bands.obj
 0002:00001918       ??_C@_0O@KLAKGGMH@code_flags_lo@ 000000018000f918     bands.obj
 0002:00001928       ??_C@_0BA@OFJPMBMN@code_attr_count@ 000000018000f928     bands.obj
 0002:00001938       ??_C@_0BC@BKACNFKP@code_attr_indexes@ 000000018000f938     bands.obj
 0002:00001950       ??_C@_0BA@DLHLCFBA@code_attr_calls@ 000000018000f950     bands.obj
 0002:00001960       ??_C@_0BF@FNGGAIBD@code_StackMapTable_N@ 000000018000f960     bands.obj
 0002:00001978       ??_C@_0BL@IJLKAPMG@code_StackMapTable_frame_T@ 000000018000f978     bands.obj
 0002:00001998       ??_C@_0BL@FLGOBHFL@code_StackMapTable_local_N@ 000000018000f998     bands.obj
 0002:000019b8       ??_C@_0BL@DBPDDGDK@code_StackMapTable_stack_N@ 000000018000f9b8     bands.obj
 0002:000019d8       ??_C@_0BK@HMGLLHPP@code_StackMapTable_offset@ 000000018000f9d8     bands.obj
 0002:000019f8       ??_C@_0BF@ONELPCMI@code_StackMapTable_T@ 000000018000f9f8     bands.obj
 0002:00001a10       ??_C@_0BG@EKILGBAE@code_StackMapTable_RC@ 000000018000fa10     bands.obj
 0002:00001a28       ??_C@_0BF@IJCHDHMM@code_StackMapTable_P@ 000000018000fa28     bands.obj
 0002:00001a40       ??_C@_0BH@EMJOIADC@code_LineNumberTable_N@ 000000018000fa40     bands.obj
 0002:00001a58       ??_C@_0BL@BODGMFAF@code_LineNumberTable_bci_P@ 000000018000fa58     bands.obj
 0002:00001a78       ??_C@_0BK@KMDHKKJP@code_LineNumberTable_line@ 000000018000fa78     bands.obj
 0002:00001a98       ??_C@_0BK@EAEINMEG@code_LocalVariableTable_N@ 000000018000fa98     bands.obj
 0002:00001ab8       ??_C@_0BO@EBBJALKI@code_LocalVariableTable_bci_P@ 000000018000fab8     bands.obj
 0002:00001ad8       ??_C@_0BP@JIPNBFGM@code_LocalVariableTable_span_O@ 000000018000fad8     bands.obj
 0002:00001af8       ??_C@_0CA@LBKLALLO@code_LocalVariableTable_name_RU@ 000000018000faf8     bands.obj
 0002:00001b18       ??_C@_0CA@OBPDECDH@code_LocalVariableTable_type_RS@ 000000018000fb18     bands.obj
 0002:00001b38       ??_C@_0BN@BAELGOA@code_LocalVariableTable_slot@ 000000018000fb38     bands.obj
 0002:00001b58       ??_C@_0BO@HHCIFDPC@code_LocalVariableTypeTable_N@ 000000018000fb58     bands.obj
 0002:00001b78       ??_C@_0CC@OECAEAHA@code_LocalVariableTypeTable_bci@ 000000018000fb78     bands.obj
 0002:00001ba0       ??_C@_0CD@BAFAHGMB@code_LocalVariableTypeTable_spa@ 000000018000fba0     bands.obj
 0002:00001bc8       ??_C@_0CE@BJEEHJII@code_LocalVariableTypeTable_nam@ 000000018000fbc8     bands.obj
 0002:00001bf0       ??_C@_0CE@EJBMDAAB@code_LocalVariableTypeTable_typ@ 000000018000fbf0     bands.obj
 0002:00001c18       ??_C@_0CB@DCPKAFMH@code_LocalVariableTypeTable_slo@ 000000018000fc18     bands.obj
 0002:00001c40       ??_C@_0BA@FEDNGPIG@code_attr_bands@ 000000018000fc40     bands.obj
 0002:00001c50       ??_C@_08ILNCKCLH@bc_codes@ 000000018000fc50     bands.obj
 0002:00001c60       ??_C@_0O@NHDHOKJ@bc_case_count@ 000000018000fc60     bands.obj
 0002:00001c70       ??_C@_0O@IPODCEHE@bc_case_value@ 000000018000fc70     bands.obj
 0002:00001c80       ??_C@_07PBCCPPFP@bc_byte@  000000018000fc80     bands.obj
 0002:00001c88       ??_C@_08LLANNIAP@bc_short@ 000000018000fc88     bands.obj
 0002:00001c98       ??_C@_08CNAAIOJJ@bc_local@ 000000018000fc98     bands.obj
 0002:00001ca8       ??_C@_08CNIFPPEB@bc_label@ 000000018000fca8     bands.obj
 0002:00001cb8       ??_C@_09LMIAJDCB@bc_intref@ 000000018000fcb8     bands.obj
 0002:00001cc8       ??_C@_0M@GHNOKACA@bc_floatref@ 000000018000fcc8     bands.obj
 0002:00001cd8       ??_C@_0L@FECALBEM@bc_longref@ 000000018000fcd8     bands.obj
 0002:00001ce8       ??_C@_0N@BLIIPDNE@bc_doubleref@ 000000018000fce8     bands.obj
 0002:00001cf8       ??_C@_0N@MPKFBKGB@bc_stringref@ 000000018000fcf8     bands.obj
 0002:00001d08       ??_C@_0BE@JPNLPCGD@bc_loadablevalueref@ 000000018000fd08     bands.obj
 0002:00001d20       ??_C@_0M@IBEIOBLC@bc_classref@ 000000018000fd20     bands.obj
 0002:00001d30       ??_C@_0M@FHDAHFFG@bc_fieldref@ 000000018000fd30     bands.obj
 0002:00001d40       ??_C@_0N@KBJNFGEO@bc_methodref@ 000000018000fd40     bands.obj
 0002:00001d50       ??_C@_0O@BOILABNA@bc_imethodref@ 000000018000fd50     bands.obj
 0002:00001d60       ??_C@_0L@MEPMLOBJ@bc_indyref@ 000000018000fd60     bands.obj
 0002:00001d70       ??_C@_0N@CGLIFEKH@bc_thisfield@ 000000018000fd70     bands.obj
 0002:00001d80       ??_C@_0O@NMPFAKNK@bc_superfield@ 000000018000fd80     bands.obj
 0002:00001d90       ??_C@_0O@OCHHHCLJ@bc_thismethod@ 000000018000fd90     bands.obj
 0002:00001da0       ??_C@_0P@MMDJDCGG@bc_supermethod@ 000000018000fda0     bands.obj
 0002:00001db0       ??_C@_0L@IAPCGJHG@bc_initref@ 000000018000fdb0     bands.obj
 0002:00001dc0       ??_C@_09BGKIKDIC@bc_escref@ 000000018000fdc0     bands.obj
 0002:00001dd0       ??_C@_0O@LHNEEOML@bc_escrefsize@ 000000018000fdd0     bands.obj
 0002:00001de0       ??_C@_0L@HJKABJFB@bc_escsize@ 000000018000fde0     bands.obj
 0002:00001df0       ??_C@_0L@HOKHNNPG@bc_escbyte@ 000000018000fdf0     bands.obj
 0002:00001e00       ??_C@_09GOEDCGAO@file_name@ 000000018000fe00     bands.obj
 0002:00001e10       ??_C@_0N@INICLDFG@file_size_hi@ 000000018000fe10     bands.obj
 0002:00001e20       ??_C@_0N@NMNBLMAM@file_size_lo@ 000000018000fe20     bands.obj
 0002:00001e30       ??_C@_0N@JMABFCDG@file_modtime@ 000000018000fe30     bands.obj
 0002:00001e40       ??_C@_0N@OPKBLMJG@file_options@ 000000018000fe40     bands.obj
 0002:00001e50       ??_C@_08FPGGDHDD@no?5index@ 000000018000fe50     bands.obj
 0002:00001e60       ??_C@_08CHILEFNK@null?5ref@ 000000018000fe60     bands.obj
 0002:00001e70       ??_C@_07MLPLAPLE@bad?5ref@ 000000018000fe70     bands.obj
 0002:00001e78       ??_C@_0BC@CJBOIHCG@overflow?5detected@ 000000018000fe78     bands.obj
 0002:00001e90       ??_C@_0BJ@CALEAGEE@Native?5allocation?5failed@ 000000018000fe90     bytes.obj
 0002:00001ec8       ??_C@_0BA@MMOCMGFH@bad?5value?5count@ 000000018000fec8     coding.obj
 0002:00001ed8       ??_C@_0L@FLIJCFOD@bad?5coding@ 000000018000fed8     coding.obj
 0002:00001ee8       ??_C@_0BE@IIPOPKNG@illegal?5arb?4?5coding@ 000000018000fee8     coding.obj
 0002:00001f00       ??_C@_0BF@OEPDPLDN@illegal?5run?5encoding@ 000000018000ff00     coding.obj
 0002:00001f18       ??_C@_0BM@FJMGNNPG@illegal?5nested?5run?5encoding@ 000000018000ff18     coding.obj
 0002:00001f38       ??_C@_0BF@JOAAKECG@illegal?5pop?5encoding@ 000000018000ff38     coding.obj
 0002:00001f50       ??_C@_0BM@CDDFICON@illegal?5nested?5pop?5encoding@ 000000018000ff50     coding.obj
 0002:00001f70       ??_C@_0BG@HLIJPJNL@pop?4L?5value?5too?5small@ 000000018000ff70     coding.obj
 0002:00001f88       ??_C@_0BH@OCEIAIEJ@pop?5token?5out?5of?5range@ 000000018000ff88     coding.obj
 0002:00001fa0       ??_C@_0CA@HBCNKKJO@bad?5meta?9coding?5for?5empty?5pop?1U@ 000000018000ffa0     coding.obj
 0002:00001fc0       ??_C@_0BA@DAENMACF@bad?5meta?9coding@ 000000018000ffc0     coding.obj
 0002:00001fd0       ??_C@_0P@DHEBFDOP@Internal?5error@ 000000018000ffd0     jni.obj
 0002:00001fe0       ??_C@_01LELAEKIP@J@        000000018000ffe0     jni.obj
 0002:00001fe8       ??_C@_0M@ODCCEGO@unpackerPtr@ 000000018000ffe8     jni.obj
 0002:00001ff8       ??_C@_0BK@MGOECGMC@cannot?5init?5class?5members@ 000000018000fff8     jni.obj
 0002:00002018       ??_C@_0BF@LHBAMMHC@?$CI?$CJLjava?1lang?1Object?$DL@ 0000000180010018     jni.obj
 0002:00002030       ??_C@_0BA@HNJNGCPJ@currentInstance@ 0000000180010030     jni.obj
 0002:00002040       ??_C@_0BK@KNKPMLAB@?$CILjava?1nio?1ByteBuffer?$DLJ?$CJJ@ 0000000180010040     jni.obj
 0002:00002060       ??_C@_0M@OOANKPPH@readInputFn@ 0000000180010060     jni.obj
 0002:0000206c       ??_C@_03IGDHHNNC@?$CI?$CJJ@ 000000018001006c     jni.obj
 0002:00002070       ??_C@_0P@BBAJIHLB@getUnpackerPtr@ 0000000180010070     jni.obj
 0002:000020b8       ??_C@_02DPKJAMEF@?$CFd@    00000001800100b8     unpack.obj
 0002:000020c0       ??_C@_0BC@DHBHLEDC@bad?5utf8?5encoding@ 00000001800100c0     unpack.obj
 0002:000020d8       ??_C@_08MPEBFEBH@bad?5data@ 00000001800100d8     unpack.obj
 0002:000020e8       ??_C@_0BI@MCADJHPK@missing?5class?5reference@ 00000001800100e8     unpack.obj
 0002:00002100       ??_C@_0BJ@DINDGABB@Internal?5buffer?5overflow@ 0000000180010100     unpack.obj
 0002:00002120       ??_C@_0BE@NBGJPKOJ@too?5much?5read?9ahead@ 0000000180010120     unpack.obj
 0002:00002138       ??_C@_0CB@MBENKFPE@EOF?5reading?5archive?5magic?5numbe@ 0000000180010138     unpack.obj
 0002:00002160       ??_C@_0CF@INONBKGM@encountered?5a?5JAR?5header?5in?5unp@ 0000000180010160     unpack.obj
 0002:00002190       ??_C@_0GN@MIAOKBBJ@?$EACorrupted?5pack?5file?3?5magic?1ver@ 0000000180010190     unpack.obj
 0002:00002200       ??_C@_0DJ@EOFNCHGA@Format?5bits?5for?5Java?57?5must?5be?5@ 0000000180010200     unpack.obj
 0002:00002240       ??_C@_0DH@PDJEDCEA@High?5archive?5option?5bits?5are?5re@ 0000000180010240     unpack.obj
 0002:00002278       ??_C@_0BP@CKGMAJKP@EOF?5reading?5fixed?5input?5buffer@ 0000000180010278     unpack.obj
 0002:00002298       ??_C@_0BI@EDJMKDIH@impossible?5archive?5size@ 0000000180010298     unpack.obj
 0002:000022b0       ??_C@_0DE@HNNKIDEL@cannot?5allocate?5large?5input?5buf@ 00000001800102b0     unpack.obj
 0002:000022e8       ??_C@_0BL@KOJPDLNM@EOF?5reading?5archive?5header@ 00000001800102e8     unpack.obj
 0002:00002308       ??_C@_0BJ@HODOOMDO@EOF?5reading?5band?5headers@ 0000000180010308     unpack.obj
 0002:00002328       ??_C@_0DB@HCOAOCOI@archive?5too?5large?3?5?5constant?5po@ 0000000180010328     unpack.obj
 0002:00002360       ??_C@_0BA@BMKLBFBL@bad?5utf8?5suffix@ 0000000180010360     unpack.obj
 0002:00002370       ??_C@_0BA@HHOGEFOO@bad?5utf8?5prefix@ 0000000180010370     unpack.obj
 0002:00002380       ??_C@_0BF@HNBIPEII@utf8?5prefix?5overflow@ 0000000180010380     unpack.obj
 0002:00002398       ??_C@_0BE@INMEHPDO@unexpected?5band?5?$CFs?6@ 0000000180010398     unpack.obj
 0002:000023b0       ??_C@_0BKA@JMJPKLFN@01?$AASignature?$AADeprecated?$AARuntime@ 00000001800103b0     unpack.obj
 0002:00002550       ??_C@_0BK@NOGBJPAL@attribute?5index?5too?5large@ 0000000180010550     unpack.obj
 0002:00002570       ??_C@_0BK@OFNJKMED@redefined?5attribute?5index@ 0000000180010570     unpack.obj
 0002:00002590       ??_C@_0BJ@OGDEGNBN@garbage?5at?5end?5of?5layout@ 0000000180010590     unpack.obj
 0002:000025b0       ??_C@_0BN@NJCEKHIO@garbage?5mixed?5with?5callables@ 00000001800105b0     unpack.obj
 0002:000025d0       ??_C@_0BD@BJONMNHI@bad?5call?5in?5layout@ 00000001800105d0     unpack.obj
 0002:000025e8       ??_C@_0BD@EOHIHJFP@bad?5layout?5element@ 00000001800105e8     unpack.obj
 0002:00002600       ??_C@_0BK@CHPLBKBJ@missing?5numeral?5in?5layout@ 0000000180010600     unpack.obj
 0002:0000261a       ??_C@_00CNPNBAHC@@         000000018001061a     unpack.obj
 0002:00002620       ??_C@_0BB@FJJKEHGJ@numeral?5overflow@ 0000000180010620     unpack.obj
 0002:00002638       ??_C@_0P@HDHNKEAB@bad?5union?5case@ 0000000180010638     unpack.obj
 0002:00002648       ??_C@_0DD@PGOJPNFL@bad?5range?5in?5union?5case?5label?5?$CI@ 0000000180010648     unpack.obj
 0002:00002680       ??_C@_0BO@JELFCPB@bad?5range?5in?5union?5case?5label@ 0000000180010680     unpack.obj
 0002:000026a0       ??_C@_0P@KBKJHJBF@bad?5case?5label@ 00000001800106a0     unpack.obj
 0002:000026b0       ??_C@_0P@MNJPOPJO@bad?5call?5label@ 00000001800106b0     unpack.obj
 0002:000026c0       ??_C@_0BF@ILAEDGAO@bad?5reference?5layout@ 00000001800106c0     unpack.obj
 0002:000026d8       ??_C@_0BE@NGGDBALG@bad?5nested?5callable@ 00000001800106d8     unpack.obj
 0002:000026f0       ??_C@_0L@FLEMDFJG@bad?5layout@ 00000001800106f0     unpack.obj
 0002:00002700       ??_C@_0JK@BMMFGJDP@?$FLNB?$FL?$CI1?$CJ?$FN?$FN?$FLNH?$FL?$CI1?$CJ?$FN?$FN?$FLRSHNH?$FLRUH?$CI1?$CJ@ 0000000180010700     unpack.obj
 0002:000027a0       ??_C@_09MAEOCCFN@?$FLNB?$FL?$CI1?$CJ?$FN?$FN@ 00000001800107a0     unpack.obj
 0002:000027b0       ??_C@_0CC@PCCOCALL@?$FLNB?$FL?$CI1?$CJ?$FN?$FN?$FLNH?$FL?$CI1?$CJ?$FN?$FN?$FLRSHNH?$FLRUH?$CI1?$CJ@ 00000001800107b0     unpack.obj
 0002:000027e0       ??_C@_0BBL@GCIMMLOG@?$FLNH?$FL?$CI1?$CJ?$CI2?$CJ?$CI3?$CJ?$FN?$FN?$FLTB?$CI0?01?$CJ?$FLB?$FN?$CI16?$CJ?$FL@ 00000001800107e0     unpack.obj
 0002:00002900       ??_C@_0BK@CIMGHPDJ@RuntimeVisibleAnnotations@ 0000000180010900     unpack.obj
 0002:00002920       ??_C@_0BM@BNNGFNMF@RuntimeInvisibleAnnotations@ 0000000180010920     unpack.obj
 0002:00002940       ??_C@_0CD@ONLIBICP@RuntimeVisibleParameterAnnotati@ 0000000180010940     unpack.obj
 0002:00002968       ??_C@_0CF@BFEAEHFK@RuntimeInvisibleParameterAnnota@ 0000000180010968     unpack.obj
 0002:00002990       ??_C@_0BC@DAGIEPHG@AnnotationDefault@ 0000000180010990     unpack.obj
 0002:000029a8       ??_C@_0BO@IJLELCEA@RuntimeVisibleTypeAnnotations@ 00000001800109a8     unpack.obj
 0002:000029c8       ??_C@_0CA@GCLMFPKD@RuntimeInvisibleTypeAnnotations@ 00000001800109c8     unpack.obj
 0002:000029e8       ??_C@_0BG@FDJMCAOP@identical?5inner?5class@ 00000001800109e8     unpack.obj
 0002:00002a00       ??_C@_0BN@GFADPNEE@undefined?5attribute?5flag?5bit@ 0000000180010a00     unpack.obj
 0002:00002a20       ??_C@_0BO@CMGKNLIA@attribute?5index?5out?5of?5bounds@ 0000000180010a20     unpack.obj
 0002:00002a40       ??_C@_0DH@OHIKFIJI@undefined?5StackMapTable?5attribu@ 0000000180010a40     unpack.obj
 0002:00002a78       ??_C@_0CL@CLGKHLIF@layout_definition?5pointer?5must?5@ 0000000180010a78     unpack.obj
 0002:00002aa8       ??_C@_0CE@NENNCDNJ@putlayout?3?5unexpected?5NULL?5for?5@ 0000000180010aa8     unpack.obj
 0002:00002ad0       ??_C@_0BB@HNCAJEIE@cp?5utf8?5overflow@ 0000000180010ad0     unpack.obj
 0002:00002ae8       ??_C@_0BC@IJJDHGHN@cp?5class?5overflow@ 0000000180010ae8     unpack.obj
 0002:00002b00       ??_C@_0BE@DAFJFMML@unpack?4deflate?4hint@ 0000000180010b00     unpack.obj
 0002:00002b18       ??_C@_0DC@KGJOKPLE@com?4sun?4java?4util?4jar?4pack?4unpa@ 0000000180010b18     unpack.obj
 0002:00002b50       ??_C@_0CD@CEMFBAGC@com?4sun?4java?4util?4jar?4pack?4verb@ 0000000180010b50     unpack.obj
 0002:00002b78       ??_C@_0DE@FNJPLIMN@com?4sun?4java?4util?4jar?4pack?4unpa@ 0000000180010b78     unpack.obj
 0002:00002bb0       ??_C@_0CL@JFLJFCLE@com?4sun?4java?4util?4jar?4pack?4unpa@ 0000000180010bb0     unpack.obj
 0002:00002bdc       ??_C@_04LKOEDJLC@keep@     0000000180010bdc     unpack.obj
 0002:00002be8       ??_C@_0CJ@LFNCLCEP@com?4sun?4java?4util?4jar?4pack?4verb@ 0000000180010be8     unpack.obj
 0002:00002c14       ??_C@_03CGLHMDPP@now@      0000000180010c14     unpack.obj
 0002:00002c18       ??_C@_01JOAMLHOP@?9@       0000000180010c18     unpack.obj
 0002:00002c20       ??_C@_0BB@MNFIFPBF@bad?5KQ?5reference@ 0000000180010c20     unpack.obj
 0002:00002c38       ??_C@_0L@PDBBHOGB@bad?5bcimap@ 0000000180010c38     unpack.obj
 0002:00002c48       ??_C@_0BM@GPDDEOEP@too?5many?5InnerClasses?5attrs@ 0000000180010c48     unpack.obj
 0002:00002c64       ??_C@_05PBJILJE@?4java@    0000000180010c64     unpack.obj
 0002:00002c70       ??_C@_0BB@MICPNADP@bad?5layout?5index@ 0000000180010c70     unpack.obj
 0002:00002c88       ??_C@_0BE@BKLBLMJK@bad?5attribute?5index@ 0000000180010c88     unpack.obj
 0002:00002ca0       ??_C@_0BN@CLDGGNCI@bad?5reference?5to?5inner?5class@ 0000000180010ca0     unpack.obj
 0002:00002cc0       ??_C@_0CC@IOEIADGN@archive?5header?5had?5incorrect?5si@ 0000000180010cc0     unpack.obj
 0002:00002ce8       ??_C@_0BM@NDDMOHPH@class?5file?5size?5transmitted@ 0000000180010ce8     unpack.obj
 0002:00002d04       ??_C@_06POIMOJKC@?4class@  0000000180010d04     unpack.obj
 0002:00002d0c       ??_C@_02DPNLHKJD@a?$CL@    0000000180010d0c     unpack.obj
 0002:00002d10       ??_C@_0BK@NDLGHGBM@Can?5not?5open?5log?5file?5?$CFs?6@ 0000000180010d10     unpack.obj
 0002:00002d30       ??_C@_0BI@CELHNJPG@error?5unpacking?5archive@ 0000000180010d30     unpack.obj
 0002:00002d50       __xmm@00000000000000ab00000001000000aa 0000000180010d50     unpack.obj
 0002:00002d60       __xmm@00000001000000a00000000700000096 0000000180010d60     unpack.obj
 0002:00002d70       ??_C@_0CE@HLJAOJEP@corrupt?5pack?5file?5or?5internal?5e@ 0000000180010d70     utils.obj
 0002:00002d98       ??_C@_0BF@JFFKOPFD@Error?3?5unpacker?3?5?$CFs?6@ 0000000180010d98     utils.obj
 0002:00002db0       ??_C@_0CG@HFNCMKIN@Error?3?5unpacker?3?5no?5current?5ins@ 0000000180010db0     utils.obj
 0002:00002de8       _pDefaultRawDllMain        0000000180010de8     MSVCRT:dll_dllmain.obj
 0002:00002de8       _pRawDllMain               0000000180010de8     MSVCRT:dll_dllmain.obj
 0002:00002e08       ??_7exception@std@@6B@     0000000180010e08     MSVCRT:throw_bad_alloc.obj
 0002:00002e18       ??_C@_0BC@EOODALEL@Unknown?5exception@ 0000000180010e18     MSVCRT:throw_bad_alloc.obj
 0002:00002e38       ??_7bad_alloc@std@@6B@     0000000180010e38     MSVCRT:throw_bad_alloc.obj
 0002:00002e48       ??_C@_0P@GHFPNOJB@bad?5allocation@ 0000000180010e48     MSVCRT:throw_bad_alloc.obj
 0002:00002e60       ??_7bad_array_new_length@std@@6B@ 0000000180010e60     MSVCRT:throw_bad_alloc.obj
 0002:00002e70       ??_C@_0BF@KINCDENJ@bad?5array?5new?5length@ 0000000180010e70     MSVCRT:throw_bad_alloc.obj
 0002:00002e90       __xmm@ffffffffffffffffffffffffffffffff 0000000180010e90     MSVCRT:utility.obj
 0002:00002ea8       ??_7type_info@@6B@         0000000180010ea8     MSVCRT:std_type_info_static.obj
 0002:00002eb0       _load_config_used          0000000180010eb0     MSVCRT:loadcfg.obj
 0002:00003080       ??_R4exception@std@@6B@    0000000180011080     MSVCRT:throw_bad_alloc.obj
 0002:000030a8       ??_R3exception@std@@8      00000001800110a8     MSVCRT:throw_bad_alloc.obj
 0002:000030c0       ??_R2exception@std@@8      00000001800110c0     MSVCRT:throw_bad_alloc.obj
 0002:000030d0       ??_R1A@?0A@EA@exception@std@@8 00000001800110d0     MSVCRT:throw_bad_alloc.obj
 0002:000030f8       ??_R4bad_alloc@std@@6B@    00000001800110f8     MSVCRT:throw_bad_alloc.obj
 0002:00003120       ??_R3bad_alloc@std@@8      0000000180011120     MSVCRT:throw_bad_alloc.obj
 0002:00003138       ??_R2bad_alloc@std@@8      0000000180011138     MSVCRT:throw_bad_alloc.obj
 0002:00003150       ??_R1A@?0A@EA@bad_alloc@std@@8 0000000180011150     MSVCRT:throw_bad_alloc.obj
 0002:00003178       ??_R4bad_array_new_length@std@@6B@ 0000000180011178     MSVCRT:throw_bad_alloc.obj
 0002:000031a0       ??_R3bad_array_new_length@std@@8 00000001800111a0     MSVCRT:throw_bad_alloc.obj
 0002:000031b8       ??_R2bad_array_new_length@std@@8 00000001800111b8     MSVCRT:throw_bad_alloc.obj
 0002:000031d8       ??_R1A@?0A@EA@bad_array_new_length@std@@8 00000001800111d8     MSVCRT:throw_bad_alloc.obj
 0002:00003200       ??_R4type_info@@6B@        0000000180011200     MSVCRT:std_type_info_static.obj
 0002:00003228       ??_R3type_info@@8          0000000180011228     MSVCRT:std_type_info_static.obj
 0002:00003240       ??_R2type_info@@8          0000000180011240     MSVCRT:std_type_info_static.obj
 0002:00003250       ??_R1A@?0A@EA@type_info@@8 0000000180011250     MSVCRT:std_type_info_static.obj
 0002:00003274       __volatile_metadata        0000000180011274     <linker-defined>
 0002:000035e8       __rtc_iaa                  00000001800115e8     MSVCRT:initsect.obj
 0002:000035f0       __rtc_izz                  00000001800115f0     MSVCRT:initsect.obj
 0002:000035f8       __rtc_taa                  00000001800115f8     MSVCRT:initsect.obj
 0002:00003600       __rtc_tzz                  0000000180011600     MSVCRT:initsect.obj
 0002:00003c28       _TI2?AVbad_alloc@std@@     0000000180011c28     MSVCRT:throw_bad_alloc.obj
 0002:00003c48       _CTA2?AVbad_alloc@std@@    0000000180011c48     MSVCRT:throw_bad_alloc.obj
 0002:00003c60       _CT??_R0?AVbad_alloc@std@@@8??0bad_alloc@std@@QEAA@AEBV01@@Z24 0000000180011c60     MSVCRT:throw_bad_alloc.obj
 0002:00003c88       _CT??_R0?AVexception@std@@@8??0exception@std@@QEAA@AEBV01@@Z24 0000000180011c88     MSVCRT:throw_bad_alloc.obj
 0002:00003cb0       _TI3?AVbad_array_new_length@std@@ 0000000180011cb0     MSVCRT:throw_bad_alloc.obj
 0002:00003cd0       _CTA3?AVbad_array_new_length@std@@ 0000000180011cd0     MSVCRT:throw_bad_alloc.obj
 0002:00003cf0       _CT??_R0?AVbad_array_new_length@std@@@8??0bad_array_new_length@std@@QEAA@AEBV01@@Z24 0000000180011cf0     MSVCRT:throw_bad_alloc.obj
 0002:00003f18       __IMPORT_DESCRIPTOR_jvm    0000000180011f18     jvm:jvm.dll
 0002:00003f2c       __IMPORT_DESCRIPTOR_java   0000000180011f2c     java:java.dll
 0002:00003f40       __IMPORT_DESCRIPTOR_KERNEL32 0000000180011f40     kernel32:KERNEL32.dll
 0002:00003f54       __IMPORT_DESCRIPTOR_VCRUNTIME140 0000000180011f54     vcruntime:VCRUNTIME140.dll
 0002:00003f68       __IMPORT_DESCRIPTOR_api-ms-win-crt-heap-l1-1-0 0000000180011f68     ucrt:api-ms-win-crt-heap-l1-1-0.dll
 0002:00003f7c       __IMPORT_DESCRIPTOR_api-ms-win-crt-stdio-l1-1-0 0000000180011f7c     ucrt:api-ms-win-crt-stdio-l1-1-0.dll
 0002:00003f90       __IMPORT_DESCRIPTOR_api-ms-win-crt-string-l1-1-0 0000000180011f90     ucrt:api-ms-win-crt-string-l1-1-0.dll
 0002:00003fa4       __IMPORT_DESCRIPTOR_api-ms-win-crt-utility-l1-1-0 0000000180011fa4     ucrt:api-ms-win-crt-utility-l1-1-0.dll
 0002:00003fb8       __IMPORT_DESCRIPTOR_api-ms-win-crt-convert-l1-1-0 0000000180011fb8     ucrt:api-ms-win-crt-convert-l1-1-0.dll
 0002:00003fcc       __IMPORT_DESCRIPTOR_api-ms-win-crt-time-l1-1-0 0000000180011fcc     ucrt:api-ms-win-crt-time-l1-1-0.dll
 0002:00003fe0       __IMPORT_DESCRIPTOR_api-ms-win-crt-runtime-l1-1-0 0000000180011fe0     ucrt:api-ms-win-crt-runtime-l1-1-0.dll
 0002:00003ff4       __NULL_IMPORT_DESCRIPTOR   0000000180011ff4     jvm:jvm.dll
 0003:00000000       ?basic_codings@@3PAUcoding@@A 0000000180013000     coding.obj
 0003:00000b00       __security_cookie_complement 0000000180013b00     MSVCRT:gs_cookie.obj
 0003:00000b08       __security_cookie          0000000180013b08     MSVCRT:gs_cookie.obj
 0003:00000b10       __scrt_native_dllmain_reason 0000000180013b10     MSVCRT:utility.obj
 0003:00000b18       __isa_available            0000000180013b18     MSVCRT:cpu_disp.obj
 0003:00000b1c       __isa_enabled              0000000180013b1c     MSVCRT:cpu_disp.obj
 0003:00000b20       __memset_fast_string_threshold 0000000180013b20     MSVCRT:cpu_disp.obj
 0003:00000b28       __memset_nt_threshold      0000000180013b28     MSVCRT:cpu_disp.obj
 0003:00000b30       __scrt_ucrt_dll_is_in_use  0000000180013b30     MSVCRT:ucrt_stubs.obj
 0003:00000b38       ??_R0?AVbad_alloc@std@@@8  0000000180013b38     MSVCRT:throw_bad_alloc.obj
 0003:00000b60       ??_R0?AVexception@std@@@8  0000000180013b60     MSVCRT:throw_bad_alloc.obj
 0003:00000b88       ??_R0?AVbad_array_new_length@std@@@8 0000000180013b88     MSVCRT:throw_bad_alloc.obj
 0003:00000bb8       ??_R0?AVtype_info@@@8      0000000180013bb8     MSVCRT:std_type_info_static.obj
 0003:00001010       ?_OptionsStorage@?1??__local_stdio_printf_options@@9@4_KA 0000000180014010     unpack.obj
 0003:000015a0       ?__type_info_root_node@@3U__type_info_node@@A 00000001800145a0     MSVCRT:tncleanup.obj
 0003:000015b0       ?_OptionsStorage@?1??__local_stdio_scanf_options@@9@4_KA 00000001800145b0     MSVCRT:default_local_stdio_options.obj
 0003:000015b8       __scrt_current_native_startup_state 00000001800145b8     MSVCRT:utility.obj
 0003:000015c0       __scrt_native_startup_lock 00000001800145c0     MSVCRT:utility.obj
 0003:00001600       __scrt_debugger_hook_flag  0000000180014600     MSVCRT:utility_desktop.obj
 0003:00001604       __favor                    0000000180014604     MSVCRT:cpu_disp.obj
 0003:00001608       __dyn_tls_init_callback    0000000180014608     <common>

 entry point at        0001:0000bf80

 Static symbols

 0000:fffe8000       .debug$S                   0000000180000000     unpack.exp
 0000:fffe8000       .debug$S                   0000000180000000     vcruntime:VCRUNTIME140.dll
 0000:fffe8000       .debug$S                   0000000180000000     vcruntime:VCRUNTIME140.dll
 0000:fffe8000       .debug$S                   0000000180000000     vcruntime:VCRUNTIME140.dll
 0000:fffe8000       .debug$S                   0000000180000000     vcruntime:VCRUNTIME140.dll
 0000:fffe8000       .debug$S                   0000000180000000     vcruntime:VCRUNTIME140.dll
 0000:fffe8000       .debug$S                   0000000180000000     vcruntime:VCRUNTIME140.dll
 0000:fffe8000       .debug$S                   0000000180000000     vcruntime:VCRUNTIME140.dll
 0000:fffe8000       .debug$S                   0000000180000000     vcruntime:VCRUNTIME140.dll
 0000:fffe8000       .debug$S                   0000000180000000     vcruntime:VCRUNTIME140.dll
 0000:fffe8000       .debug$S                   0000000180000000     vcruntime:VCRUNTIME140.dll
 0000:fffe8000       .debug$S                   0000000180000000     vcruntime:VCRUNTIME140.dll
 0000:fffe8000       .debug$S                   0000000180000000     vcruntime:VCRUNTIME140.dll
 0000:fffe8000       .debug$S                   0000000180000000     vcruntime:VCRUNTIME140.dll
 0000:fffe8000       .debug$S                   0000000180000000     ucrt:api-ms-win-crt-convert-l1-1-0.dll
 0000:fffe8000       .debug$S                   0000000180000000     ucrt:api-ms-win-crt-filesystem-l1-1-0.dll
 0002:ffff2000       .idata$6                   0000000180000000     ucrt:api-ms-win-crt-filesystem-l1-1-0.dll
 0000:fffe8000       .debug$S                   0000000180000000     ucrt:api-ms-win-crt-heap-l1-1-0.dll
 0000:fffe8000       .debug$S                   0000000180000000     ucrt:api-ms-win-crt-heap-l1-1-0.dll
 0000:fffe8000       .debug$S                   0000000180000000     ucrt:api-ms-win-crt-heap-l1-1-0.dll
 0000:fffe8000       .debug$S                   0000000180000000     ucrt:api-ms-win-crt-heap-l1-1-0.dll
 0000:fffe8000       .debug$S                   0000000180000000     ucrt:api-ms-win-crt-heap-l1-1-0.dll
 0000:fffe8000       .debug$S                   0000000180000000     ucrt:api-ms-win-crt-runtime-l1-1-0.dll
 0000:fffe8000       .debug$S                   0000000180000000     ucrt:api-ms-win-crt-runtime-l1-1-0.dll
 0000:fffe8000       .debug$S                   0000000180000000     ucrt:api-ms-win-crt-runtime-l1-1-0.dll
 0000:fffe8000       .debug$S                   0000000180000000     ucrt:api-ms-win-crt-runtime-l1-1-0.dll
 0000:fffe8000       .debug$S                   0000000180000000     ucrt:api-ms-win-crt-runtime-l1-1-0.dll
 0000:fffe8000       .debug$S                   0000000180000000     ucrt:api-ms-win-crt-runtime-l1-1-0.dll
 0000:fffe8000       .debug$S                   0000000180000000     ucrt:api-ms-win-crt-runtime-l1-1-0.dll
 0000:fffe8000       .debug$S                   0000000180000000     ucrt:api-ms-win-crt-runtime-l1-1-0.dll
 0000:fffe8000       .debug$S                   0000000180000000     ucrt:api-ms-win-crt-runtime-l1-1-0.dll
 0000:fffe8000       .debug$S                   0000000180000000     ucrt:api-ms-win-crt-runtime-l1-1-0.dll
 0000:fffe8000       .debug$S                   0000000180000000     ucrt:api-ms-win-crt-runtime-l1-1-0.dll
 0000:fffe8000       .debug$S                   0000000180000000     ucrt:api-ms-win-crt-runtime-l1-1-0.dll
 0000:fffe8000       .debug$S                   0000000180000000     ucrt:api-ms-win-crt-runtime-l1-1-0.dll
 0000:fffe8000       .debug$S                   0000000180000000     ucrt:api-ms-win-crt-runtime-l1-1-0.dll
 0000:fffe8000       .debug$S                   0000000180000000     ucrt:api-ms-win-crt-runtime-l1-1-0.dll
 0000:fffe8000       .debug$S                   0000000180000000     ucrt:api-ms-win-crt-stdio-l1-1-0.dll
 0000:fffe8000       .debug$S                   0000000180000000     ucrt:api-ms-win-crt-stdio-l1-1-0.dll
 0000:fffe8000       .debug$S                   0000000180000000     ucrt:api-ms-win-crt-stdio-l1-1-0.dll
 0000:fffe8000       .debug$S                   0000000180000000     ucrt:api-ms-win-crt-stdio-l1-1-0.dll
 0000:fffe8000       .debug$S                   0000000180000000     ucrt:api-ms-win-crt-stdio-l1-1-0.dll
 0000:fffe8000       .debug$S                   0000000180000000     ucrt:api-ms-win-crt-stdio-l1-1-0.dll
 0000:fffe8000       .debug$S                   0000000180000000     ucrt:api-ms-win-crt-stdio-l1-1-0.dll
 0000:fffe8000       .debug$S                   0000000180000000     ucrt:api-ms-win-crt-string-l1-1-0.dll
 0000:fffe8000       .debug$S                   0000000180000000     ucrt:api-ms-win-crt-string-l1-1-0.dll
 0000:fffe8000       .debug$S                   0000000180000000     ucrt:api-ms-win-crt-string-l1-1-0.dll
 0000:fffe8000       .debug$S                   0000000180000000     ucrt:api-ms-win-crt-string-l1-1-0.dll
 0000:fffe8000       .debug$S                   0000000180000000     ucrt:api-ms-win-crt-string-l1-1-0.dll
 0000:fffe8000       .debug$S                   0000000180000000     ucrt:api-ms-win-crt-time-l1-1-0.dll
 0000:fffe8000       .debug$S                   0000000180000000     ucrt:api-ms-win-crt-time-l1-1-0.dll
 0000:fffe8000       .debug$S                   0000000180000000     ucrt:api-ms-win-crt-utility-l1-1-0.dll
 0000:fffe8000       .debug$S                   0000000180000000     kernel32:KERNEL32.dll
 0000:fffe8000       .debug$S                   0000000180000000     kernel32:KERNEL32.dll
 0000:fffe8000       .debug$S                   0000000180000000     kernel32:KERNEL32.dll
 0000:fffe8000       .debug$S                   0000000180000000     kernel32:KERNEL32.dll
 0000:fffe8000       .debug$S                   0000000180000000     kernel32:KERNEL32.dll
 0000:fffe8000       .debug$S                   0000000180000000     kernel32:KERNEL32.dll
 0000:fffe8000       .debug$S                   0000000180000000     kernel32:KERNEL32.dll
 0000:fffe8000       .debug$S                   0000000180000000     kernel32:KERNEL32.dll
 0000:fffe8000       .debug$S                   0000000180000000     kernel32:KERNEL32.dll
 0000:fffe8000       .debug$S                   0000000180000000     kernel32:KERNEL32.dll
 0000:fffe8000       .debug$S                   0000000180000000     kernel32:KERNEL32.dll
 0000:fffe8000       .debug$S                   0000000180000000     kernel32:KERNEL32.dll
 0000:fffe8000       .debug$S                   0000000180000000     kernel32:KERNEL32.dll
 0000:fffe8000       .debug$S                   0000000180000000     kernel32:KERNEL32.dll
 0000:fffe8000       .debug$S                   0000000180000000     kernel32:KERNEL32.dll
 0000:fffe8000       .debug$S                   0000000180000000     kernel32:KERNEL32.dll
 0000:fffe8000       .debug$S                   0000000180000000     kernel32:KERNEL32.dll
 0000:fffe8000       .debug$S                   0000000180000000     jvm:jvm.dll
 0000:fffe8000       .debug$S                   0000000180000000     java:java.dll
 0001:00001a94       ?get_unpacker@@YAPEAUunpacker@@PEAUJNIEnv_@@PEAV_jobject@@_N@Z 0000000180002a94 f   jni.obj
 0001:00001b5c       ?get_unpacker@@YAPEAUunpacker@@XZ 0000000180002b5c f   jni.obj
 0001:00001c0c       ?read_input_via_jni@@YA_JPEAUunpacker@@PEAX_J2@Z 0000000180002c0c f   jni.obj
 0001:0000279c       ?compare_Utf8_chars@@YAHAEAUbytes@@0@Z 000000018000379c f   unpack.obj
 0001:00009330       ?store_Utf8_char@@YAPEACPEACG@Z 000000018000a330 f   unpack.obj
 0001:0000bb80       $$000000                   000000018000cb80     MSVCRT:amdsecgs.obj
 0001:0000bc00       $$000000                   000000018000cc00     MSVCRT:chkstk.obj
 0001:0000bc60       ?dllmain_crt_dispatch@@YAHQEAUHINSTANCE__@@KQEAX@Z 000000018000cc60 f   MSVCRT:dll_dllmain.obj
 0001:0000bcb0       ?dllmain_crt_process_attach@@YAHQEAUHINSTANCE__@@QEAX@Z 000000018000ccb0 f   MSVCRT:dll_dllmain.obj
 0001:0000bdc8       ?dllmain_crt_process_detach@@YAH_N@Z 000000018000cdc8 f   MSVCRT:dll_dllmain.obj
 0001:0000be4c       ?dllmain_dispatch@@YAHQEAUHINSTANCE__@@KQEAX@Z 000000018000ce4c f   MSVCRT:dll_dllmain.obj
 0001:0000c0c8       capture_previous_context   000000018000d0c8 f   MSVCRT:gs_report.obj
 0001:0000cb80       $$000000                   000000018000db80     MSVCRT:guard_dispatch.obj
 0001:0000cba0       $$000000                   000000018000dba0     MSVCRT:guard_xfg_dispatch.obj
 0001:0000cbb6       ?fin$0@?0??dllmain_crt_process_attach@@YAHQEAUHINSTANCE__@@QEAX@Z@4HA 000000018000dbb6 f   MSVCRT:dll_dllmain.obj
 0001:0000cbcd       ?fin$0@?0??dllmain_crt_process_detach@@YAH_N@Z@4HA 000000018000dbcd f   MSVCRT:dll_dllmain.obj
 0001:0000cbe6       ?fin$1@?0??dllmain_crt_process_detach@@YAH_N@Z@4HA 000000018000dbe6 f   MSVCRT:dll_dllmain.obj
 0001:0000cbfa       ?filt$0@?0??dllmain_dispatch@@YAHQEAUHINSTANCE__@@KQEAX@Z@4HA 000000018000dbfa f   MSVCRT:dll_dllmain.obj
 0001:0000cc30       __scrt_is_nonwritable_in_current_image$filt$0 000000018000dc30 f   MSVCRT:utility.obj
 0002:00000270       ?all_band_inits@@3QBUband_init@@B 000000018000e270     bands.obj
 0002:00001eb0       ?ERB@@3QBDB                000000018000feb0     coding.obj
 0002:00002080       ?TAG_ORDER@@3QBCB          0000000180010080     unpack.obj
 0002:00002098       ?str_tf@@3QBDB             0000000180010098     unpack.obj
 0002:000020a8       ?TAGS_IN_ORDER@@3QBCB      00000001800100a8     unpack.obj
 0002:00002dd8       ?jarmagic@@3QBGB           0000000180010dd8     zip.obj
 0002:00002de0       ?marker_comment@@3QBDB     0000000180010de0     zip.obj
 0002:00002df0       GS_ExceptionPointers       0000000180010df0     MSVCRT:gs_report.obj
 0002:00003608       $unwind$?readData@band@@QEAAXH@Z 0000000180011608     bands.obj
 0002:00003628       $unwind$?getRefCommon@band@@QEAAPEAUentry@@PEAUcpindex@@_N@Z 0000000180011628     bands.obj
 0002:00003628       $unwind$?getInt@value_stream@@QEAAHXZ 0000000180011628     coding.obj
 0002:00003628       $unwind$?get_unpacker@@YAPEAUunpacker@@PEAUJNIEnv_@@PEAV_jobject@@_N@Z 0000000180011628     jni.obj
 0002:00003628       $unwind$Java_com_sun_java_util_jar_pack_NativeUnpack_finish 0000000180011628     jni.obj
 0002:00003628       $unwind$Java_com_sun_java_util_jar_pack_NativeUnpack_getNextFile 0000000180011628     jni.obj
 0002:00003628       $unwind$Java_com_sun_java_util_jar_pack_NativeUnpack_getOption 0000000180011628     jni.obj
 0002:00003628       $unwind$?ensure_input@unpacker@@QEAA_N_J@Z 0000000180011628     unpack.obj
 0002:00003628       $unwind$?free@unpacker@@QEAAXXZ 0000000180011628     unpack.obj
 0002:00003628       $unwind$?readBandData@attr_definitions@unpacker@@QEAAXH@Z 0000000180011628     unpack.obj
 0002:00003628       $unwind$?requestOutputIndex@entry@@QEAAXAEAUcpool@@H@Z 0000000180011628     unpack.obj
 0002:00003628       $unwind$__scrt_dllmain_exception_filter 0000000180011628     MSVCRT:utility.obj
 0002:0000363c       $unwind$?getLong@band@@QEAA_JAEAU1@_N@Z 000000018001163c     bands.obj
 0002:0000363c       $unwind$?freeAll@ptrlist@@QEAAXXZ 000000018001163c     bytes.obj
 0002:0000363c       $unwind$?realloc@bytes@@QEAAX_K@Z 000000018001163c     bytes.obj
 0002:0000363c       $unwind$?saveFrom@bytes@@QEAAXPEBX_K@Z 000000018001163c     bytes.obj
 0002:0000363c       $unwind$?computeOutputIndexes@cpool@@QEAAXXZ 000000018001163c     unpack.obj
 0002:0000363c       $unwind$?ensure_put_space@unpacker@@QEAAX_K@Z 000000018001163c     unpack.obj
 0002:0000363c       $unwind$?put_label@unpacker@@QEAAXHH@Z 000000018001163c     unpack.obj
 0002:0000363c       $unwind$?putref_index@unpacker@@QEAAHPEAUentry@@H@Z 000000018001163c     unpack.obj
 0002:0000363c       $unwind$?read_classes@unpacker@@QEAAXXZ 000000018001163c     unpack.obj
 0002:0000363c       $unwind$?read_files@unpacker@@QEAAXXZ 000000018001163c     unpack.obj
 0002:0000363c       $unwind$?redirect_stdio@unpacker@@QEAAXXZ 000000018001163c     unpack.obj
 0002:0000363c       $unwind$_DllMainCRTStartup 000000018001163c     MSVCRT:dll_dllmain.obj
 0002:0000364c       $unwind$?getIntTotal@band@@QEAAHXZ 000000018001164c     bands.obj
 0002:0000364c       $unwind$Java_com_sun_java_util_jar_pack_NativeUnpack_start 000000018001164c     jni.obj
 0002:0000364c       $unwind$?buildBands@attr_definitions@unpacker@@QEAAPEAPEAUband@@PEAUlayout_definition@2@@Z 000000018001164c     unpack.obj
 0002:0000364c       $unwind$?calloc_heap@unpacker@@QEAAPEAX_K0_N1@Z 000000018001164c     unpack.obj
 0002:00003664       $unwind$?getIntCount@band@@QEAAHH@Z 0000000180011664     bands.obj
 0002:00003664       $unwind$?makeBands@band@@SAPEAU1@PEAUunpacker@@@Z 0000000180011664     bands.obj
 0002:00003664       $unwind$?get_next_file@unpacker@@QEAAPEAUfile@1@XZ 0000000180011664     unpack.obj
 0002:0000367c       $unwind$?free@bytes@@QEAAXXZ 000000018001167c     bytes.obj
 0002:0000367c       $unwind$?malloc@bytes@@QEAAX_K@Z 000000018001167c     bytes.obj
 0002:0000367c       $unwind$?setCoding@value_stream@@QEAAXPEAUcoding@@@Z 000000018001167c     coding.obj
 0002:0000367c       $unwind$?getKQIndex@cpool@@QEAAPEAUcpindex@@XZ 000000018001167c     unpack.obj
 0002:0000367c       $unwind$?putu2@unpacker@@QEAAXH@Z 000000018001167c     unpack.obj
 0002:0000367c       $unwind$?putu4@unpacker@@QEAAXH@Z 000000018001167c     unpack.obj
 0002:0000367c       $unwind$?putu8@unpacker@@QEAAX_J@Z 000000018001167c     unpack.obj
 0002:0000367c       $unwind$?read_bands@unpacker@@QEAAXXZ 000000018001167c     unpack.obj
 0002:0000367c       $unwind$?reset_cur_classfile@unpacker@@QEAAXXZ 000000018001167c     unpack.obj
 0002:0000367c       $unwind$?must_calloc@@YAPEAX_K0@Z 000000018001167c     utils.obj
 0002:0000367c       $unwind$?unpack_abort@@YAXPEBDPEAUunpacker@@@Z 000000018001167c     utils.obj
 0002:0000367c       $unwind$__raise_securityfailure 000000018001167c     MSVCRT:gs_report.obj
 0002:0000367c       $unwind$??2@YAPEAX_K@Z     000000018001167c     MSVCRT:new_scalar.obj
 0002:0000367c       $unwind$??_Gtype_info@@UEAAPEAXI@Z 000000018001167c     MSVCRT:std_type_info_static.obj
 0002:0000367c       $unwind$??0bad_alloc@std@@QEAA@AEBV01@@Z 000000018001167c     MSVCRT:throw_bad_alloc.obj
 0002:0000367c       $unwind$??0bad_array_new_length@std@@QEAA@AEBV01@@Z 000000018001167c     MSVCRT:throw_bad_alloc.obj
 0002:0000367c       $unwind$??0exception@std@@QEAA@AEBV01@@Z 000000018001167c     MSVCRT:throw_bad_alloc.obj
 0002:0000367c       $unwind$__scrt_initialize_crt 000000018001167c     MSVCRT:utility.obj
 0002:0000367c       $unwind$__scrt_initialize_onexit_tables 000000018001167c     MSVCRT:utility.obj
 0002:0000367c       $unwind$__scrt_release_startup_lock 000000018001167c     MSVCRT:utility.obj
 0002:0000367c       $unwind$__scrt_uninitialize_crt 000000018001167c     MSVCRT:utility.obj
 0002:00003684       $unwind$?compareTo@bytes@@QEAAHAEAU1@@Z 0000000180011684     bytes.obj
 0002:00003684       $unwind$?ensureSize@fillbytes@@QEAAX_K@Z 0000000180011684     bytes.obj
 0002:00003684       $unwind$?writeTo@bytes@@QEAAPEACPEAC@Z 0000000180011684     bytes.obj
 0002:00003684       $unwind$?findBySpec@coding@@SAPEAU1@H@Z 0000000180011684     coding.obj
 0002:00003684       $unwind$Java_com_sun_java_util_jar_pack_NativeUnpack_initIDs 0000000180011684     jni.obj
 0002:00003684       $unwind$?free@attr_definitions@unpacker@@QEAAXXZ 0000000180011684     unpack.obj
 0002:00003684       $unwind$?parseNumeral@attr_definitions@unpacker@@QEAAPEBDPEBDAEAH@Z 0000000180011684     unpack.obj
 0002:00003684       $unwind$?put_space@unpacker@@QEAAPEAC_K@Z 0000000180011684     unpack.obj
 0002:00003684       $unwind$?put_stackmap_type@unpacker@@QEAAXXZ 0000000180011684     unpack.obj
 0002:00003684       $unwind$?putref@unpacker@@QEAAXPEAUentry@@@Z 0000000180011684     unpack.obj
 0002:00003684       $unwind$?putu1ref@unpacker@@QEAAXPEAUentry@@@Z 0000000180011684     unpack.obj
 0002:00003684       $unwind$?typeSize@entry@@QEAAHXZ 0000000180011684     unpack.obj
 0002:00003684       $unwind$?init@jar@@QEAAXPEAUunpacker@@@Z 0000000180011684     zip.obj
 0002:00003684       $unwind$_RTC_Initialize    0000000180011684     MSVCRT:initsect.obj
 0002:00003684       $unwind$_RTC_Terminate     0000000180011684     MSVCRT:initsect.obj
 0002:00003684       $unwind$??_Gbad_alloc@std@@UEAAPEAXI@Z 0000000180011684     MSVCRT:throw_bad_alloc.obj
 0002:00003684       $unwind$??_Gbad_array_new_length@std@@UEAAPEAXI@Z 0000000180011684     MSVCRT:throw_bad_alloc.obj
 0002:00003684       $unwind$??_Gexception@std@@UEAAPEAXI@Z 0000000180011684     MSVCRT:throw_bad_alloc.obj
 0002:00003690       $unwind$?grow@fillbytes@@QEAAPEAC_K@Z 0000000180011690     bytes.obj
 0002:00003690       $unwind$?saveTo@unpacker@@QEAAXAEAUbytes@@PEAC_K@Z 0000000180011690     unpack.obj
 0002:000036a4       $unwind$?init@coding@@QEAAPEAU1@XZ 00000001800116a4     coding.obj
 0002:000036a4       $unwind$?get_code_header@unpacker@@QEAAXAEAH000@Z 00000001800116a4     unpack.obj
 0002:000036b8       $unwind$?parse@coding@@SAIAEAPEACHH@Z 00000001800116b8     coding.obj
 0002:000036b8       $unwind$?parse_lgH@coding@@SAIAEAPEACHHH@Z 00000001800116b8     coding.obj
 0002:000036c8       $unwind$?parseMultiple@coding@@SAXAEAPEACHPEACHH@Z 00000001800116c8     coding.obj
 0002:000036c8       $unwind$__GSHandlerCheckCommon 00000001800116c8     MSVCRT:gshandler.obj
 0002:000036d0       $unwind$?init@coding_method@@QEAAXAEAPEACPEAC0HPEAUcoding@@HPEAUintlist@@@Z 00000001800116d0     coding.obj
 0002:000036f0       $unwind$?CallLongMethod@JNIEnv_@@QEAA_JPEAV_jobject@@PEAU_jmethodID@@ZZ 00000001800116f0     jni.obj
 0002:000036f0       $unwind$?CallStaticObjectMethod@JNIEnv_@@QEAAPEAV_jobject@@PEAV_jclass@@PEAU_jmethodID@@ZZ 00000001800116f0     jni.obj
 0002:000036f8       $unwind$Java_com_sun_java_util_jar_pack_NativeUnpack_getUnusedInput 00000001800116f8     jni.obj
 0002:000036f8       $unwind$?abort@unpacker@@QEAAXPEBD@Z 00000001800116f8     unpack.obj
 0002:000036f8       $unwind$?init@unpacker@@QEAAXP6A_JPEAU1@PEAX_J2@Z@Z 00000001800116f8     unpack.obj
 0002:000036f8       $unwind$?initGroupIndexes@cpool@@QEAAXXZ 00000001800116f8     unpack.obj
 0002:00003704       $unwind$Java_com_sun_java_util_jar_pack_NativeUnpack_setOption 0000000180011704     jni.obj
 0002:00003704       $unwind$?write_classfile_head@unpacker@@QEAAXXZ 0000000180011704     unpack.obj
 0002:00003704       $unwind$?write_classfile_tail@unpacker@@QEAAXXZ 0000000180011704     unpack.obj
 0002:0000371c       $unwind$?read_input_via_jni@@YA_JPEAUunpacker@@PEAX_J2@Z 000000018001171c     jni.obj
 0002:0000371c       $unwind$?init@cpool@@QEAAXPEAUunpacker@@QEAH@Z 000000018001171c     unpack.obj
 0002:0000371c       $unwind$?popBody@attr_definitions@unpacker@@QEAAPEAPEAUband@@H@Z 000000018001171c     unpack.obj
 0002:0000372c       $unwind$?get_unpacker@@YAPEAUunpacker@@XZ 000000018001172c     jni.obj
 0002:00003738       $unwind$fprintf            0000000180011738     unpack.obj
 0002:00003738       $unwind$sprintf            0000000180011738     unpack.obj
 0002:00003744       $unwind$_snprintf          0000000180011744     unpack.obj
 0002:00003754       $unwind$?hashTabRef@cpool@@QEAAAEAPEAUentry@@CAEAUbytes@@@Z 0000000180011754     unpack.obj
 0002:00003770       $unwind$?ensureUtf8@cpool@@QEAAPEAUentry@@AEAUbytes@@@Z 0000000180011770     unpack.obj
 0002:00003784       $unwind$?ensureClass@cpool@@QEAAPEAUentry@@AEAUbytes@@@Z 0000000180011784     unpack.obj
 0002:00003798       $unwind$?expandSignatures@cpool@@QEAAXXZ 0000000180011798     unpack.obj
 0002:000037b0       $unwind$?initMemberIndexes@cpool@@QEAAXXZ 00000001800117b0     unpack.obj
 0002:000037c8       $unwind$?defineLayout@attr_definitions@unpacker@@QEAAPEAUlayout_definition@2@HPEBD0@Z 00000001800117c8     unpack.obj
 0002:000037e0       $unwind$?parseLayout@attr_definitions@unpacker@@QEAAPEBDPEBDAEAPEAPEAUband@@H@Z 00000001800117e0     unpack.obj
 0002:000037f8       $unwind$?parseIntLayout@attr_definitions@unpacker@@QEAAPEBDPEBDAEAPEAUband@@C_N@Z 00000001800117f8     unpack.obj
 0002:00003814       $unwind$?readBandData@attr_definitions@unpacker@@QEAAXPEAPEAUband@@I@Z 0000000180011814     unpack.obj
 0002:0000382c       $unwind$?set_option@unpacker@@QEAA_NPEBD0@Z 000000018001182c     unpack.obj
 0002:00003840       $unwind$?get_option@unpacker@@QEAAPEBDPEBD@Z 0000000180011840     unpack.obj
 0002:00003858       $unwind$?start@unpacker@@QEAAXPEAX_K@Z 0000000180011858     unpack.obj
 0002:00003858       $unwind$?to_bci@unpacker@@QEAAII@Z 0000000180011858     unpack.obj
 0002:00003858       $unwind$?unpack_aborting@@YA_NPEAUunpacker@@@Z 0000000180011858     utils.obj
 0002:00003858       $unwind$__scrt_initialize_default_local_stdio_options 0000000180011858     MSVCRT:default_local_stdio_options.obj
 0002:00003858       $unwind$?dllmain_crt_dispatch@@YAHQEAUHINSTANCE__@@KQEAX@Z 0000000180011858     MSVCRT:dll_dllmain.obj
 0002:00003858       $unwind$DllMain            0000000180011858     MSVCRT:dll_dllmain_stub.obj
 0002:00003858       $unwind$__GSHandlerCheck   0000000180011858     MSVCRT:gshandler.obj
 0002:00003858       $unwind$__scrt_acquire_startup_lock 0000000180011858     MSVCRT:utility.obj
 0002:00003858       $unwind$__scrt_dllmain_after_initialize_c 0000000180011858     MSVCRT:utility.obj
 0002:00003858       $unwind$__scrt_dllmain_before_initialize_c 0000000180011858     MSVCRT:utility.obj
 0002:00003858       $unwind$__scrt_dllmain_crt_thread_attach 0000000180011858     MSVCRT:utility.obj
 0002:00003858       $unwind$__scrt_dllmain_crt_thread_detach 0000000180011858     MSVCRT:utility.obj
 0002:00003858       $unwind$__scrt_dllmain_uninitialize_c 0000000180011858     MSVCRT:utility.obj
 0002:00003858       $unwind$__scrt_dllmain_uninitialize_critical 0000000180011858     MSVCRT:utility.obj
 0002:00003860       $unwind$?checkLegacy@unpacker@@QEAAXPEBD@Z 0000000180011860     unpack.obj
 0002:00003874       $unwind$?putlayout@unpacker@@QEAAXPEAPEAUband@@@Z 0000000180011874     unpack.obj
 0002:00003890       $unwind$?write_code@unpacker@@QEAAXXZ 0000000180011890     unpack.obj
 0002:000038a0       $unwind$?write_bc_ops@unpacker@@QEAAXXZ 00000001800118a0     unpack.obj
 0002:000038b8       $unwind$?write_members@unpacker@@QEAAXHH@Z 00000001800118b8     unpack.obj
 0002:000038d0       $unwind$?write_attrs@unpacker@@QEAAHH_K@Z 00000001800118d0     unpack.obj
 0002:000038f4       $unwind$?write_ics@unpacker@@QEAAHHH@Z 00000001800118f4     unpack.obj
 0002:00003910       $unwind$?write_bsms@unpacker@@QEAAHHH@Z 0000000180011910     unpack.obj
 0002:0000392c       $unwind$?read_file_header@unpacker@@QEAAXXZ 000000018001192c     unpack.obj
 0002:00003954       $unwind$?read_cp@unpacker@@QEAAXXZ 0000000180011954     unpack.obj
 0002:0000396c       $unwind$?read_attr_defs@unpacker@@QEAAXXZ 000000018001196c     unpack.obj
 0002:00003988       $unwind$?read_ics@unpacker@@QEAAXXZ 0000000180011988     unpack.obj
 0002:000039a4       $unwind$?read_attrs@unpacker@@QEAAXHH@Z 00000001800119a4     unpack.obj
 0002:000039bc       $unwind$?read_code_headers@unpacker@@QEAAXXZ 00000001800119bc     unpack.obj
 0002:000039cc       $unwind$?read_bcs@unpacker@@QEAAXXZ 00000001800119cc     unpack.obj
 0002:000039e4       $unwind$?read_Utf8_values@unpacker@@QEAAXPEAUentry@@HC@Z 00000001800119e4     unpack.obj
 0002:000039fc       $unwind$?read_single_words@unpacker@@QEAAXAEAUband@@PEAUentry@@HCH@Z 00000001800119fc     unpack.obj
 0002:00003a18       $unwind$?read_double_words@unpacker@@QEAAXAEAUband@@PEAUentry@@HCH@Z 0000000180011a18     unpack.obj
 0002:00003a30       $unwind$?read_single_refs@unpacker@@QEAAXAEAUband@@CPEAUentry@@HCH@Z 0000000180011a30     unpack.obj
 0002:00003a48       $unwind$?read_double_refs@unpacker@@QEAAXAEAUband@@CCPEAUentry@@HC@Z 0000000180011a48     unpack.obj
 0002:00003a60       $unwind$?read_signature_values@unpacker@@QEAAXPEAUentry@@HC@Z 0000000180011a60     unpack.obj
 0002:00003a7c       $unwind$?read_method_handle@unpacker@@QEAAXPEAUentry@@HCH@Z 0000000180011a7c     unpack.obj
 0002:00003a7c       $unwind$?read_method_type@unpacker@@QEAAXPEAUentry@@HCH@Z 0000000180011a7c     unpack.obj
 0002:00003a98       $unwind$?read_bootstrap_methods@unpacker@@QEAAXPEAUentry@@HC@Z 0000000180011a98     unpack.obj
 0002:00003ab4       $unwind$?compare_Utf8_chars@@YAHAEAUbytes@@0@Z 0000000180011ab4     unpack.obj
 0002:00003ad0       $xdatasym                  0000000180011ad0     MSVCRT:amdsecgs.obj
 0002:00003ad8       $xdatasym                  0000000180011ad8     MSVCRT:chkstk.obj
 0002:00003ae0       $unwind$?dllmain_crt_process_attach@@YAHQEAUHINSTANCE__@@QEAX@Z 0000000180011ae0     MSVCRT:dll_dllmain.obj
 0002:00003b1c       $unwind$?fin$0@?0??dllmain_crt_process_attach@@YAHQEAUHINSTANCE__@@QEAX@Z@4HA 0000000180011b1c     MSVCRT:dll_dllmain.obj
 0002:00003b1c       $unwind$?fin$0@?0??dllmain_crt_process_detach@@YAH_N@Z@4HA 0000000180011b1c     MSVCRT:dll_dllmain.obj
 0002:00003b1c       $unwind$?fin$1@?0??dllmain_crt_process_detach@@YAH_N@Z@4HA 0000000180011b1c     MSVCRT:dll_dllmain.obj
 0002:00003b24       $unwind$?dllmain_crt_process_detach@@YAH_N@Z 0000000180011b24     MSVCRT:dll_dllmain.obj
 0002:00003b78       $unwind$?dllmain_dispatch@@YAHQEAUHINSTANCE__@@KQEAX@Z 0000000180011b78     MSVCRT:dll_dllmain.obj
 0002:00003ba0       $unwind$?filt$0@?0??dllmain_dispatch@@YAHQEAUHINSTANCE__@@KQEAX@Z@4HA 0000000180011ba0     MSVCRT:dll_dllmain.obj
 0002:00003ba8       $unwind$__report_gsfailure 0000000180011ba8     MSVCRT:gs_report.obj
 0002:00003bb0       $unwind$capture_previous_context 0000000180011bb0     MSVCRT:gs_report.obj
 0002:00003bbc       $unwind$?__scrt_throw_std_bad_alloc@@YAXXZ 0000000180011bbc     MSVCRT:throw_bad_alloc.obj
 0002:00003bbc       $unwind$?__scrt_throw_std_bad_array_new_length@@YAXXZ 0000000180011bbc     MSVCRT:throw_bad_alloc.obj
 0002:00003bc4       $unwind$__security_init_cookie 0000000180011bc4     MSVCRT:gs_support.obj
 0002:00003bd0       $unwind$__scrt_is_nonwritable_in_current_image 0000000180011bd0     MSVCRT:utility.obj
 0002:00003bf0       $unwind$__scrt_is_nonwritable_in_current_image$filt$0 0000000180011bf0     MSVCRT:utility.obj
 0002:00003bf8       $unwind$__scrt_fastfail    0000000180011bf8     MSVCRT:utility_desktop.obj
 0002:00003c08       $unwind$__isa_available_init 0000000180011c08     MSVCRT:cpu_disp.obj
 0002:00003c18       $xdatasym                  0000000180011c18     MSVCRT:guard_dispatch.obj
 0002:00003c20       $xdatasym                  0000000180011c20     MSVCRT:guard_xfg_dispatch.obj
 0002:00003d20       .edata                     0000000180011d20     unpack.exp
 0002:00003d48       rgpv                       0000000180011d48     unpack.exp
 0002:00003d64       rgszName                   0000000180011d64     unpack.exp
 0002:00003d80       rgwOrd                     0000000180011d80     unpack.exp
 0002:00003d8e       szName                     0000000180011d8e     unpack.exp
 0002:00003d99       $N00001                    0000000180011d99     unpack.exp
 0002:00003dcd       $N00002                    0000000180011dcd     unpack.exp
 0002:00003e06       $N00003                    0000000180011e06     unpack.exp
 0002:00003e3d       $N00004                    0000000180011e3d     unpack.exp
 0002:00003e79       $N00005                    0000000180011e79     unpack.exp
 0002:00003eae       $N00006                    0000000180011eae     unpack.exp
 0002:00003ee5       $N00007                    0000000180011ee5     unpack.exp
 0002:00004210       .idata$6                   0000000180012210     jvm:jvm.dll
 0002:00004230       .idata$6                   0000000180012230     java:java.dll
 0002:000043a0       .idata$6                   00000001800123a0     kernel32:KERNEL32.dll
 0002:00004456       .idata$6                   0000000180012456     vcruntime:VCRUNTIME140.dll
 0002:000045d8       .idata$6                   00000001800125d8     ucrt:api-ms-win-crt-heap-l1-1-0.dll
 0002:000045f8       .idata$6                   00000001800125f8     ucrt:api-ms-win-crt-stdio-l1-1-0.dll
 0002:00004618       .idata$6                   0000000180012618     ucrt:api-ms-win-crt-string-l1-1-0.dll
 0002:0000463a       .idata$6                   000000018001263a     ucrt:api-ms-win-crt-utility-l1-1-0.dll
 0002:0000465c       .idata$6                   000000018001265c     ucrt:api-ms-win-crt-convert-l1-1-0.dll
 0002:0000467e       .idata$6                   000000018001267e     ucrt:api-ms-win-crt-time-l1-1-0.dll
 0002:0000469e       .idata$6                   000000018001269e     ucrt:api-ms-win-crt-runtime-l1-1-0.dll
 0003:00000be0       ?dummy@@3PACA              0000000180013be0     bytes.obj
 0003:00000fe0       ?no_meta@@3PAPEBCA         0000000180013fe0     coding.obj
 0003:00000fe8       ?unpackerPtrFID@@3PEAU_jfieldID@@EA 0000000180013fe8     jni.obj
 0003:00000ff0       ?currentInstMID@@3PEAU_jmethodID@@EA 0000000180013ff0     jni.obj
 0003:00000ff8       ?readInputMID@@3PEAU_jmethodID@@EA 0000000180013ff8     jni.obj
 0003:00001000       ?NIclazz@@3PEAV_jclass@@EA 0000000180014000     jni.obj
 0003:00001008       ?getUnpackerPtrMID@@3PEAU_jmethodID@@EA 0000000180014008     jni.obj
 0003:00001018       ?no_bands@@3PAPEAUband@@A  0000000180014018     unpack.obj
 0003:00001020       ?__proc_attached@@3HA      0000000180014020     MSVCRT:dll_dllmain.obj
 0003:00001030       GS_ExceptionRecord         0000000180014030     MSVCRT:gs_report.obj
 0003:000010d0       GS_ContextRecord           00000001800140d0     MSVCRT:gs_report.obj
 0003:000015c8       ?is_initialized_as_dll@@3_NA 00000001800145c8     MSVCRT:utility.obj
 0003:000015c9       ?module_local_atexit_table_initialized@@3_NA 00000001800145c9     MSVCRT:utility.obj
 0003:000015d0       ?module_local_atexit_table@@3U_onexit_table_t@@A 00000001800145d0     MSVCRT:utility.obj
 0003:000015e8       ?module_local_at_quick_exit_table@@3U_onexit_table_t@@A 00000001800145e8     MSVCRT:utility.obj
 0005:00000060       $R000000                   0000000180016060     unpack.dll.res
